 esdhc

 Timestamp is 4da2a516 (Mon Apr 11 18:52:06 2011)

 Preferred load address is 10000000

 Start         Length     Name                   Class
 0001:00000000 000044f6H .rdata                  CODE
 0001:000044f8 00000022H .rdata$debug            CODE
 0001:0000451c 0001720cH .text                   CODE
 0001:0001b728 00000068H .xdata                  CODE
 0001:0001b790 00000050H .idata$2                CODE
 0001:0001b7e0 00000014H .idata$3                CODE
 0001:0001b7f4 0000015cH .idata$4                CODE
 0001:0001b950 00000104H .idata$6                CODE
 0001:0001ba60 000000c7H .edata                  CODE
 0002:00000000 0000015cH .idata$5                DATA
 0002:00000160 00000498H .data                   DATA
 0002:000005f8 0000005cH .bss                    DATA
 0003:00000000 000008c8H .pdata                  DATA

  Address         Publics by Value              Rva+Base       Lib:Object

 0000:00000000       ___safe_se_handler_table   00000000     <absolute>
 0000:00000000       ___safe_se_handler_count   00000000     <absolute>
 0001:0000001c       ??_C@_1BM@NNIPIGOJ@?$AAW?$AAa?$AAk?$AAe?$AAu?$AAp?$AAS?$AAo?$AAu?$AAr?$AAc?$AAe?$AAs?$AA?$AA@ 1000101c     bspesdhc.obj
 0001:00000038       ??_C@_1CC@LMBBBPNF@?$AAR?$AAe?$AAa?$AAd?$AAW?$AAr?$AAi?$AAt?$AAe?$AAT?$AAi?$AAm?$AAe?$AAo?$AAu?$AAt?$AA?$AA@ 10001038     bspesdhc.obj
 0001:0000005c       ??_C@_1CM@FPPMGDBH@?$AAM?$AAa?$AAx?$AAi?$AAm?$AAu?$AAm?$AAC?$AAl?$AAo?$AAc?$AAk?$AAF?$AAr?$AAe?$AAq?$AAu?$AAe?$AAn?$AAc?$AAy?$AA?$AA@ 1000105c     bspesdhc.obj
 0001:00000088       ??_C@_1BK@KBGNDCFC@?$AAS?$AAD?$AAI?$AAO?$AAP?$AAr?$AAi?$AAo?$AAr?$AAi?$AAt?$AAy?$AA?$AA@ 10001088     bspesdhc.obj
 0001:000000a4       ??_C@_1BG@OINKPJMJ@?$AAD?$AAi?$AAs?$AAa?$AAb?$AAl?$AAe?$AAD?$AAM?$AAA?$AA?$AA@ 100010a4     bspesdhc.obj
 0001:000000c0       ??_C@_1KO@HCDMJLCG@?$AAC?$AAE?$AAS?$AAD?$AAH?$AAC?$AAB?$AAa?$AAs?$AAe?$AA?3?$AA?3?$AAG?$AAe?$AAt?$AAR?$AAe?$AAg?$AAi?$AAs?$AAt?$AAr?$AAy?$AAS?$AAe?$AAt?$AAt?$AAi?$AAn?$AAg?$AAs?$AA?3@ 100010c0     bspesdhc.obj
 0001:00000170       ??_C@_1M@EENNDIOJ@?$AAI?$AAn?$AAd?$AAe?$AAx?$AA?$AA@ 10001170     bspesdhc.obj
 0001:00000180       ??_C@_1FK@FNONLNGN@?$AA?$CF?$AAs?$AA?3?$AA?5?$AAD?$AAE?$AAB?$AAU?$AAG?$AAC?$AAH?$AAK?$AA?5?$AAf?$AAa?$AAi?$AAl?$AAe?$AAd?$AA?5?$AAi?$AAn?$AA?5?$AAf?$AAi?$AAl?$AAe?$AA?5?$AA?$CF?$AAs?$AA?5?$AAa@ 10001180     bspesdhc.obj
 0001:000001e0       ??_C@_1JG@KMJCDHON@?$AAc?$AA?3?$AA?2?$AAw?$AAi?$AAn?$AAc?$AAe?$AAr?$AAo?$AAo?$AAt?$AAs?$AA?2?$AAt?$AAo?$AAp?$AAa?$AAz?$AA?2?$AAw?$AAi?$AAn?$AAc?$AAe?$AA7?$AA0?$AA0?$AA?2?$AAp?$AAl?$AAa@ 100011e0     bspesdhc.obj
 0001:00000278       ??_7CESDHCBaseEDMA@@6B@    10001278     bspesdhcdma.obj
 0001:00000294       ??_C@_1BM@OOIHKKEA@?$AAS?$AAD?$AAH?$AAC?$AA?5?$AA?9?$AAD?$AAe?$AAi?$AAn?$AAi?$AAt?$AA?6?$AA?$AA@ 10001294     esdhcbase_common_topaz_v1:sdmain.obj
 0001:000002b0       ??_C@_1BM@OAPLBGMF@?$AAS?$AAD?$AAH?$AAC?$AA?5?$AA?$CL?$AAD?$AAe?$AAi?$AAn?$AAi?$AAt?$AA?6?$AA?$AA@ 100012b0     esdhcbase_common_topaz_v1:sdmain.obj
 0001:000002cc       ??_C@_1BI@MLPKMGB@?$AAS?$AAD?$AAH?$AAC?$AA?5?$AA?9?$AAI?$AAn?$AAi?$AAt?$AA?6?$AA?$AA@ 100012cc     esdhcbase_common_topaz_v1:sdmain.obj
 0001:000002e8       ??_C@_1FC@NPNLGMF@?$AAS?$AAD?$AAH?$AAC?$AA?5?$AAF?$AAa?$AAi?$AAl?$AAe?$AAd?$AA?5?$AAt?$AAo?$AA?5?$AAc?$AAr?$AAe?$AAa?$AAt?$AAe?$AA?5?$AAc?$AAo?$AAn?$AAt?$AAr?$AAo?$AAl?$AAl?$AAe?$AAr@ 100012e8     esdhcbase_common_topaz_v1:sdmain.obj
 0001:0000033c       ??_C@_1DE@PGNMCNJP@?$AAS?$AAD?$AAH?$AAC?$AA?5?$AAA?$AAc?$AAt?$AAi?$AAv?$AAe?$AA?5?$AAR?$AAe?$AAg?$AAP?$AAa?$AAt?$AAh?$AA?3?$AA?5?$AA?$CF?$AAs?$AA?5?$AA?6?$AA?$AA@ 1000133c     esdhcbase_common_topaz_v1:sdmain.obj
 0001:00000370       ??_C@_1BI@PEHNOHNH@?$AAS?$AAD?$AAH?$AAC?$AA?5?$AA?$CL?$AAI?$AAn?$AAi?$AAt?$AA?6?$AA?$AA@ 10001370     esdhcbase_common_topaz_v1:sdmain.obj
 0001:00000388       ??_C@_1CC@CBKGMBFG@?$AAS?$AAD?$AAH?$AAC?$AA?5?$AA?9?$AAI?$AAO?$AAC?$AAo?$AAn?$AAt?$AAr?$AAo?$AAl?$AA?6?$AA?$AA@ 10001388     esdhcbase_common_topaz_v1:sdmain.obj
 0001:000003ac       ??_C@_1CC@JBJLJDAG@?$AAS?$AAD?$AAH?$AAC?$AA?5?$AA?$CL?$AAI?$AAO?$AAC?$AAo?$AAn?$AAt?$AAr?$AAo?$AAl?$AA?6?$AA?$AA@ 100013ac     esdhcbase_common_topaz_v1:sdmain.obj
 0001:000003d0       ??_C@_1GI@OIOBLEEB@?$AAC?$AAE?$AAS?$AAD?$AAH?$AAC?$AAB?$AAa?$AAs?$AAe?$AA?3?$AA?3?$AAS?$AAe?$AAt?$AAI?$AAn?$AAt?$AAe?$AAr?$AAf?$AAa?$AAc?$AAe?$AA?3?$AA?5?$AAS?$AAe?$AAt?$AAt?$AAi?$AAn@ 100013d0     esdhcbase_common_topaz_v1:esdhc.obj
 0001:00000438       ??_C@_1GA@BJFBOADM@?$AAC?$AAE?$AAS?$AAD?$AAH?$AAC?$AAB?$AAa?$AAs?$AAe?$AA?3?$AA?3?$AAS?$AAe?$AAt?$AAI?$AAn?$AAt?$AAe?$AAr?$AAf?$AAa?$AAc?$AAe?$AA?3?$AA?5?$AAP?$AAR?$AAO?$AAC?$AAT?$AAL@ 10001438     esdhcbase_common_topaz_v1:esdhc.obj
 0001:00000498       ??_C@_1GG@MCMMKGOO@?$AAC?$AAE?$AAS?$AAD?$AAH?$AAC?$AAB?$AAa?$AAs?$AAe?$AA?3?$AA?3?$AAS?$AAe?$AAt?$AAI?$AAn?$AAt?$AAe?$AAr?$AAf?$AAa?$AAc?$AAe?$AA?3?$AA?5?$AAS?$AAe?$AAt?$AAt?$AAi?$AAn@ 10001498     esdhcbase_common_topaz_v1:esdhc.obj
 0001:00000500       ??_C@_1KK@LKKGEGCK@?$AAc?$AA?3?$AA?2?$AAw?$AAi?$AAn?$AAc?$AAe?$AAr?$AAo?$AAo?$AAt?$AAs?$AA?2?$AAt?$AAo?$AAp?$AAa?$AAz?$AA?2?$AAw?$AAi?$AAn?$AAc?$AAe?$AA7?$AA0?$AA0?$AA?2?$AAp?$AAl?$AAa@ 10001500     esdhcbase_common_topaz_v1:esdhc.obj
 0001:000005b0       ??_C@_1EI@HHLEBCDF@?$AA?$CL?$AAC?$AAE?$AAS?$AAD?$AAH?$AAC?$AAS?$AAl?$AAo?$AAt?$AA?3?$AA?3?$AAE?$AAn?$AAa?$AAb?$AAl?$AAe?$AAS?$AAD?$AAI?$AAO?$AAI?$AAn?$AAt?$AAe?$AAr?$AAr?$AAu?$AAp?$AAt@ 100015b0     esdhcbase_common_topaz_v1:esdhc.obj
 0001:000005f8       ??_C@_1EK@LFKJGIHP@?$AA?$CL?$AAC?$AAE?$AAS?$AAD?$AAH?$AAC?$AAS?$AAl?$AAo?$AAt?$AA?3?$AA?3?$AAD?$AAi?$AAs?$AAa?$AAb?$AAl?$AAe?$AAS?$AAD?$AAI?$AAO?$AAI?$AAn?$AAt?$AAe?$AAr?$AAr?$AAu?$AAp@ 100015f8     esdhcbase_common_topaz_v1:esdhc.obj
 0001:00000648       ??_C@_1IC@JDDBOGML@?$AAS?$AAe?$AAt?$AAC?$AAl?$AAo?$AAc?$AAk?$AAR?$AAa?$AAt?$AAe?$AA?5?$AA?9?$AA?5?$AAR?$AAe?$AAq?$AAu?$AAe?$AAs?$AAt?$AAe?$AAd?$AA?5?$AAR?$AAa?$AAt?$AAe?$AA?3?$AA?5?$AA?$CF@ 10001648     esdhcbase_common_topaz_v1:esdhc.obj
 0001:000006d0       ??_C@_1OM@MFDMGGNM@?$AAC?$AAE?$AAS?$AAD?$AAH?$AAC?$AAB?$AAa?$AAs?$AAe?$AA?3?$AA?3?$AAS?$AAe?$AAn?$AAd?$AAC?$AAo?$AAm?$AAm?$AAa?$AAn?$AAd?$AA?3?$AA?5?$AAC?$AAm?$AAd?$AA?5?$AA?$DN?$AA?5?$AA0@ 100016d0     esdhcbase_common_topaz_v1:esdhc.obj
 0001:000007c0       ??_C@_1FO@PFNBHMHH@?$AAS?$AAe?$AAn?$AAd?$AAC?$AAo?$AAm?$AAm?$AAa?$AAn?$AAd?$AA?3?$AA?5?$AAC?$AAD?$AAI?$AAH?$AAB?$AA?5?$AAs?$AAe?$AAt?$AA?4?$AA?5?$AAC?$AAa?$AAn?$AAn?$AAo?$AAt?$AA?5?$AAs@ 100017c0     esdhcbase_common_topaz_v1:esdhc.obj
 0001:00000820       ??_C@_1FM@MDDIBGAF@?$AAS?$AAe?$AAn?$AAd?$AAC?$AAo?$AAm?$AAm?$AAa?$AAn?$AAd?$AA?3?$AA?5?$AAC?$AAI?$AAH?$AAB?$AA?5?$AAs?$AAe?$AAt?$AA?4?$AA?5?$AAC?$AAa?$AAn?$AAn?$AAo?$AAt?$AA?5?$AAs?$AAe@ 10001820     esdhcbase_common_topaz_v1:esdhc.obj
 0001:00000880       ??_C@_1GC@IHNGGPKM@?$AAS?$AAe?$AAn?$AAd?$AAC?$AAo?$AAm?$AAm?$AAa?$AAn?$AAd?$AA?3?$AA?5?$AAA?$AAu?$AAt?$AAo?$AAC?$AAM?$AAD?$AA1?$AA2?$AA?5?$AAS?$AAu?$AAc?$AAc?$AAe?$AAe?$AAd?$AAe?$AAd@ 10001880     esdhcbase_common_topaz_v1:esdhc.obj
 0001:000008e8       ??_C@_1MI@DEHLPGLK@?$AAC?$AAE?$AAS?$AAD?$AAH?$AAC?$AAB?$AAa?$AAs?$AAe?$AA?3?$AA?3?$AAH?$AAa?$AAn?$AAd?$AAl?$AAe?$AAR?$AAe?$AAm?$AAo?$AAv?$AAa?$AAl?$AA?3?$AA?5?$AAC?$AAa?$AAr?$AAd?$AA?5@ 100018e8     esdhcbase_common_topaz_v1:esdhc.obj
 0001:000009b0       ??_C@_1BO@JHAGCEDM@?$AA?7?$AA?5?$AAH?$AAC?$AAP?$AAa?$AAr?$AAa?$AAm?$AA?3?$AA?5?$AA?$CF?$AAd?$AA?6?$AA?$AA@ 100019b0     esdhcbase_common_topaz_v1:esdhc.obj
 0001:000009d0       ??_C@_1CC@FBIHCMNE@?$AA?7?$AA?5?$AAB?$AAl?$AAo?$AAc?$AAk?$AAS?$AAi?$AAz?$AAe?$AA?3?$AA?5?$AA?$CF?$AAd?$AA?6?$AA?$AA@ 100019d0     esdhcbase_common_topaz_v1:esdhc.obj
 0001:000009f4       ??_C@_1CC@GNOBEPDN@?$AA?7?$AA?5?$AAN?$AAu?$AAm?$AAB?$AAl?$AAo?$AAc?$AAk?$AAs?$AA?3?$AA?5?$AA?$CF?$AAd?$AA?6?$AA?$AA@ 100019f4     esdhcbase_common_topaz_v1:esdhc.obj
 0001:00000a18       ??_C@_1CI@CNEJOFAE@?$AA?7?$AA?5?$AAR?$AAe?$AAs?$AAp?$AAo?$AAn?$AAs?$AAe?$AAT?$AAy?$AAp?$AAe?$AA?3?$AA?5?$AA?$CF?$AAd?$AA?6?$AA?$AA@ 10001a18     esdhcbase_common_topaz_v1:esdhc.obj
 0001:00000a40       ??_C@_1CI@ODABMFDF@?$AA?7?$AA?5?$AAA?$AAr?$AAg?$AAu?$AAm?$AAe?$AAn?$AAt?$AA?3?$AA?5?$AA0?$AAx?$AA?$CF?$AA0?$AA8?$AAx?$AA?6?$AA?$AA@ 10001a40     esdhcbase_common_topaz_v1:esdhc.obj
 0001:00000a68       ??_C@_1BO@JBKIJFEK@?$AA?7?$AA?5?$AAC?$AAo?$AAm?$AAm?$AAa?$AAn?$AAd?$AA?3?$AA?5?$AA?$CF?$AAd?$AA?6?$AA?$AA@ 10001a68     esdhcbase_common_topaz_v1:esdhc.obj
 0001:00000a88       ??_C@_1DI@FBGDIKAJ@?$AAD?$AAu?$AAm?$AAp?$AAC?$AAu?$AAr?$AAr?$AAe?$AAn?$AAt?$AAR?$AAe?$AAq?$AAu?$AAe?$AAs?$AAt?$AA?3?$AA?5?$AA0?$AAx?$AA?$CF?$AA0?$AA8?$AAX?$AA?6?$AA?$AA@ 10001a88     esdhcbase_common_topaz_v1:esdhc.obj
 0001:00000ac0       ??_C@_1DO@MNDMEBDK@?$AA?$CL?$AAC?$AAE?$AAS?$AAD?$AAH?$AAC?$AAB?$AAa?$AAs?$AAe?$AA?3?$AA?3?$AAH?$AAa?$AAn?$AAd?$AAl?$AAe?$AAI?$AAn?$AAs?$AAe?$AAr?$AAt?$AAi?$AAo?$AAn?$AA?$AN?$AA?6?$AA?$AA@ 10001ac0     esdhcbase_common_topaz_v1:esdhc.obj
 0001:00000b00       ??_C@_1IO@LMIELODG@?$AAH?$AAa?$AAn?$AAd?$AAl?$AAe?$AAC?$AAo?$AAm?$AAm?$AAa?$AAn?$AAd?$AAE?$AAr?$AAr?$AAo?$AAr?$AAs?$AA?5?$AA?9?$AA?5?$AAC?$AAo?$AAm?$AAm?$AAa?$AAn?$AAd?$AA?5?$AAl?$AAi@ 10001b00     esdhcbase_common_topaz_v1:esdhc.obj
 0001:00000b90       ??_C@_1GA@FKENBLIK@?$AAH?$AAa?$AAn?$AAd?$AAl?$AAe?$AAC?$AAo?$AAm?$AAm?$AAa?$AAn?$AAd?$AAE?$AAr?$AAr?$AAo?$AAr?$AAs?$AA?5?$AA?9?$AA?5?$AAS?$AAT?$AAA?$AAT?$AAU?$AAS?$AA?5?$AAE?$AAR?$AAR@ 10001b90     esdhcbase_common_topaz_v1:esdhc.obj
 0001:00000bf0       ??_C@_1IO@IIPKGMNA@?$AAH?$AAa?$AAn?$AAd?$AAl?$AAe?$AAD?$AAa?$AAt?$AAa?$AAE?$AAr?$AAr?$AAo?$AAr?$AAs?$AA?5?$AA?9?$AA?5?$AAD?$AAa?$AAt?$AAa?$AA?5?$AAl?$AAi?$AAn?$AAe?$AA?5?$AAe?$AAr?$AAr@ 10001bf0     esdhcbase_common_topaz_v1:esdhc.obj
 0001:00000c80       ??_C@_1II@OIJDKAAP@?$AAH?$AAa?$AAn?$AAd?$AAl?$AAe?$AAD?$AAa?$AAt?$AAa?$AAE?$AAr?$AAr?$AAo?$AAr?$AAs?$AA?5?$AA?9?$AA?5?$AAI?$AAn?$AAt?$AAe?$AAr?$AAn?$AAa?$AAl?$AA?5?$AAD?$AAM?$AAA?$AA?5@ 10001c80     esdhcbase_common_topaz_v1:esdhc.obj
 0001:00000d08       ??_C@_1FK@KJKJOMID@?$AAH?$AAa?$AAn?$AAd?$AAl?$AAe?$AAD?$AAa?$AAt?$AAa?$AAE?$AAr?$AAr?$AAo?$AAr?$AAs?$AA?5?$AA?9?$AA?5?$AAS?$AAT?$AAA?$AAT?$AAU?$AAS?$AA?5?$AAE?$AAR?$AAR?$AAO?$AAR?$AA?5@ 10001d08     esdhcbase_common_topaz_v1:esdhc.obj
 0001:00000d68       ??_C@_1FA@JMEHCNIG@?$AAE?$AAx?$AAc?$AAe?$AAp?$AAt?$AAi?$AAo?$AAn?$AA?5?$AAr?$AAe?$AAa?$AAd?$AAi?$AAn?$AAg?$AA?5?$AAf?$AAr?$AAo?$AAm?$AA?5?$AAc?$AAl?$AAi?$AAe?$AAn?$AAt?$AA?5?$AAb?$AAu@ 10001d68     esdhcbase_common_topaz_v1:esdhc.obj
 0001:00000db8       ??_C@_1DO@BJDFFIMF@?$AA?$CL?$AAC?$AAE?$AAS?$AAD?$AAH?$AAC?$AAB?$AAa?$AAs?$AAe?$AA?3?$AA?3?$AAH?$AAa?$AAn?$AAd?$AAl?$AAe?$AAR?$AAe?$AAa?$AAd?$AAR?$AAe?$AAa?$AAd?$AAy?$AA?$AN?$AA?6?$AA?$AA@ 10001db8     esdhcbase_common_topaz_v1:esdhc.obj
 0001:00000df8       ??_C@_1EA@JOJFPIOB@?$AA?$CL?$AAC?$AAE?$AAS?$AAD?$AAH?$AAC?$AAB?$AAa?$AAs?$AAe?$AA?3?$AA?3?$AAH?$AAa?$AAn?$AAd?$AAl?$AAe?$AAW?$AAr?$AAi?$AAt?$AAe?$AAR?$AAe?$AAa?$AAd?$AAy?$AA?$AN?$AA?6?$AA?$AA@ 10001df8     esdhcbase_common_topaz_v1:esdhc.obj
 0001:00000e38       ??_C@_1HC@ECLLLECE@?$AAC?$AAE?$AAS?$AAD?$AAH?$AAC?$AAB?$AAa?$AAs?$AAe?$AA?3?$AA?3?$AAH?$AAa?$AAn?$AAd?$AAl?$AAe?$AAI?$AAn?$AAt?$AAe?$AAr?$AAr?$AAu?$AAp?$AAt?$AAs?$AA?3?$AA?5?$AAR?$AAe@ 10001e38     esdhcbase_common_topaz_v1:esdhc.obj
 0001:00000eac       ??_C@_1BA@LEPJIIOK@?$AAU?$AAn?$AAk?$AAn?$AAo?$AAw?$AAn?$AA?$AA@ 10001eac     esdhcbase_common_topaz_v1:esdhc.obj
 0001:00000ebc       ??_C@_1CC@NMDOMPHL@?$AAM?$AAS?$AAC?$AA_?$AAD?$AAE?$AAT?$AAA?$AAC?$AAH?$AA_?$AAE?$AAV?$AAE?$AAN?$AAT?$AA?$AA@ 10001ebc     esdhcbase_common_topaz_v1:esdhc.obj
 0001:00000ee0       ??_C@_1BG@MPOEBAN@?$AAM?$AAS?$AAC?$AA_?$AAS?$AAD?$AAD?$AAI?$AAS?$AAK?$AA?$AA@ 10001ee0     esdhcbase_common_topaz_v1:esdhc.obj
 0001:00000ef8       ??_C@_1GC@LFLKMPEO@?$AAC?$AAE?$AAS?$AAD?$AAH?$AAC?$AAS?$AAl?$AAo?$AAt?$AA?3?$AA?3?$AAH?$AAa?$AAn?$AAd?$AAl?$AAe?$AAI?$AAn?$AAt?$AAe?$AAr?$AAr?$AAu?$AAp?$AAt?$AAs?$AA?3?$AA?5?$AAC?$AAa@ 10001ef8     esdhcbase_common_topaz_v1:esdhc.obj
 0001:00000f60       ??_C@_1GE@OLACPKOF@?$AAC?$AAE?$AAS?$AAD?$AAH?$AAC?$AAS?$AAl?$AAo?$AAt?$AA?3?$AA?3?$AAH?$AAa?$AAn?$AAd?$AAl?$AAe?$AAI?$AAn?$AAt?$AAe?$AAr?$AAr?$AAu?$AAp?$AAt?$AAs?$AA?3?$AA?5?$AAC?$AAa@ 10001f60     esdhcbase_common_topaz_v1:esdhc.obj
 0001:00000fc8       ??_C@_1EA@JEBGJAHH@?$AA?$CL?$AAC?$AAE?$AAS?$AAD?$AAH?$AAC?$AAS?$AAl?$AAo?$AAt?$AA?3?$AA?3?$AAH?$AAa?$AAn?$AAd?$AAl?$AAe?$AAI?$AAn?$AAt?$AAe?$AAr?$AAr?$AAu?$AAp?$AAt?$AAs?$AA?$AN?$AA?6?$AA?$AA@ 10001fc8     esdhcbase_common_topaz_v1:esdhc.obj
 0001:00001008       ??_C@_1FE@PKPHCKKI@?$AA?9?$AAD?$AAu?$AAm?$AAp?$AAE?$AAS?$AAD?$AAH?$AAC?$AAR?$AAe?$AAg?$AAs?$AA?9?$AA?9?$AA?9?$AA?9?$AA?9?$AA?9?$AA?9?$AA?9?$AA?9?$AA?9?$AA?9?$AA?9?$AA?9?$AA?9?$AA?9?$AA?9?$AA?9?$AA?9@ 10002008     esdhcbase_common_topaz_v1:esdhc.obj
 0001:0000105c       ??_C@_1CE@HKGLJMHP@?$AAH?$AAO?$AAS?$AAT?$AAV?$AAE?$AAR?$AA?5?$AA0?$AAx?$AA?$CF?$AA0?$AA8?$AAX?$AA?5?$AA?$AN?$AA?6?$AA?$AA@ 1000205c     esdhcbase_common_topaz_v1:esdhc.obj
 0001:00001080       ??_C@_1BM@DEJEGJIL@?$AAW?$AAM?$AAL?$AA?5?$AA0?$AAx?$AA?$CF?$AA0?$AA8?$AAX?$AA?5?$AA?$AN?$AA?6?$AA?$AA@ 10002080     esdhcbase_common_topaz_v1:esdhc.obj
 0001:0000109c       ??_C@_1CK@BIIHIBDO@?$AAH?$AAO?$AAS?$AAT?$AAC?$AAA?$AAP?$AAB?$AAL?$AAT?$AA?5?$AA0?$AAx?$AA?$CF?$AA0?$AA8?$AAX?$AA?5?$AA?$AN?$AA?6?$AA?$AA@ 1000209c     esdhcbase_common_topaz_v1:esdhc.obj
 0001:000010c8       ??_C@_1CK@PPNHIOLN@?$AAA?$AAU?$AAT?$AAO?$AAC?$AA1?$AA2?$AAE?$AAR?$AAR?$AA?5?$AA0?$AAx?$AA?$CF?$AA0?$AA8?$AAX?$AA?5?$AA?$AN?$AA?6?$AA?$AA@ 100020c8     esdhcbase_common_topaz_v1:esdhc.obj
 0001:000010f4       ??_C@_1CE@JHGAFBMP@?$AAI?$AAR?$AAQ?$AAS?$AAT?$AAA?$AAT?$AA?5?$AA0?$AAx?$AA?$CF?$AA0?$AA8?$AAX?$AA?5?$AA?$AN?$AA?6?$AA?$AA@ 100020f4     esdhcbase_common_topaz_v1:esdhc.obj
 0001:00001118       ??_C@_1CC@HIONAACK@?$AAS?$AAY?$AAS?$AAC?$AAT?$AAL?$AA?5?$AA0?$AAx?$AA?$CF?$AA0?$AA8?$AAX?$AA?5?$AA?$AN?$AA?6?$AA?$AA@ 10002118     esdhcbase_common_topaz_v1:esdhc.obj
 0001:0000113c       ??_C@_1CC@IGHJGBLI@?$AAP?$AAR?$AAO?$AAC?$AAT?$AAL?$AA?5?$AA0?$AAx?$AA?$CF?$AA0?$AA8?$AAX?$AA?5?$AA?$AN?$AA?6?$AA?$AA@ 1000213c     esdhcbase_common_topaz_v1:esdhc.obj
 0001:00001160       ??_C@_1CE@KLDEFLDN@?$AAP?$AAR?$AAS?$AAS?$AAT?$AAA?$AAT?$AA?5?$AA0?$AAx?$AA?$CF?$AA0?$AA8?$AAX?$AA?5?$AA?$AN?$AA?6?$AA?$AA@ 10002160     esdhcbase_common_topaz_v1:esdhc.obj
 0001:00001184       ??_C@_1CE@DCDHMBDP@?$AAC?$AAM?$AAD?$AAR?$AAS?$AAP?$AA3?$AA?5?$AA0?$AAx?$AA?$CF?$AA0?$AA8?$AAX?$AA?5?$AA?$AN?$AA?6?$AA?$AA@ 10002184     esdhcbase_common_topaz_v1:esdhc.obj
 0001:000011a8       ??_C@_1CE@LDBCKEBI@?$AAC?$AAM?$AAD?$AAR?$AAS?$AAP?$AA2?$AA?5?$AA0?$AAx?$AA?$CF?$AA0?$AA8?$AAX?$AA?5?$AA?$AN?$AA?6?$AA?$AA@ 100021a8     esdhcbase_common_topaz_v1:esdhc.obj
 0001:000011cc       ??_C@_1CE@OLAMANDA@?$AAC?$AAM?$AAD?$AAR?$AAS?$AAP?$AA1?$AA?5?$AA0?$AAx?$AA?$CF?$AA0?$AA8?$AAX?$AA?5?$AA?$AN?$AA?6?$AA?$AA@ 100021cc     esdhcbase_common_topaz_v1:esdhc.obj
 0001:000011f0       ??_C@_1CE@GKCJGIBH@?$AAC?$AAM?$AAD?$AAR?$AAS?$AAP?$AA0?$AA?5?$AA0?$AAx?$AA?$CF?$AA0?$AA8?$AAX?$AA?5?$AA?$AN?$AA?6?$AA?$AA@ 100021f0     esdhcbase_common_topaz_v1:esdhc.obj
 0001:00001214       ??_C@_1CE@JCCAMFCN@?$AAX?$AAF?$AAE?$AAR?$AAT?$AAY?$AAP?$AA?5?$AA0?$AAx?$AA?$CF?$AA0?$AA8?$AAX?$AA?5?$AA?$AN?$AA?6?$AA?$AA@ 10002214     esdhcbase_common_topaz_v1:esdhc.obj
 0001:00001238       ??_C@_1CC@ECOAEKGN@?$AAC?$AAM?$AAD?$AAA?$AAR?$AAG?$AA?5?$AA0?$AAx?$AA?$CF?$AA0?$AA8?$AAX?$AA?5?$AA?$AN?$AA?6?$AA?$AA@ 10002238     esdhcbase_common_topaz_v1:esdhc.obj
 0001:0000125c       ??_C@_1CE@JLLLHPCC@?$AAB?$AAL?$AAK?$AAA?$AAT?$AAT?$AAR?$AA?5?$AA0?$AAx?$AA?$CF?$AA0?$AA8?$AAX?$AA?5?$AA?$AN?$AA?6?$AA?$AA@ 1000225c     esdhcbase_common_topaz_v1:esdhc.obj
 0001:00001280       ??_C@_1CC@MCCINEKA@?$AAD?$AAS?$AAA?$AAD?$AAD?$AAR?$AA?5?$AA0?$AAx?$AA?$CF?$AA0?$AA8?$AAX?$AA?5?$AA?$AN?$AA?6?$AA?$AA@ 10002280     esdhcbase_common_topaz_v1:esdhc.obj
 0001:000012a8       ??_C@_1FE@PNIPOOEL@?$AA?$CL?$AAD?$AAu?$AAm?$AAp?$AAE?$AAS?$AAD?$AAH?$AAC?$AAR?$AAe?$AAg?$AAs?$AA?9?$AA?9?$AA?9?$AA?9?$AA?9?$AA?9?$AA?9?$AA?9?$AA?9?$AA?9?$AA?9?$AA?9?$AA?9?$AA?9?$AA?9?$AA?9?$AA?9?$AA?9@ 100022a8     esdhcbase_common_topaz_v1:esdhc.obj
 0001:000012fc       ??_C@_1CI@BOJPMJKG@?$AA?9?$AAC?$AAE?$AAS?$AAD?$AAH?$AAC?$AAB?$AAa?$AAs?$AAe?$AA?3?$AA?3?$AAI?$AAn?$AAi?$AAt?$AA?$AN?$AA?6?$AA?$AA@ 100022fc     esdhcbase_common_topaz_v1:esdhc.obj
 0001:00001328       ??_C@_1HO@COFPAFLJ@?$AAC?$AAE?$AAS?$AAD?$AAH?$AAC?$AAB?$AAa?$AAs?$AAe?$AA?3?$AA?3?$AAI?$AAn?$AAi?$AAt?$AA?3?$AA?5?$AAF?$AAa?$AAi?$AAl?$AAe?$AAd?$AA?5?$AAt?$AAo?$AA?5?$AAr?$AAe?$AAg?$AAi@ 10002328     esdhcbase_common_topaz_v1:esdhc.obj
 0001:000013a8       ??_C@_1GK@JGJOACME@?$AAC?$AAE?$AAS?$AAD?$AAH?$AAC?$AAB?$AAa?$AAs?$AAe?$AA?3?$AA?3?$AAI?$AAn?$AAi?$AAt?$AA?3?$AA?5?$AAE?$AAr?$AAr?$AAo?$AAr?$AA?5?$AAa?$AAl?$AAl?$AAo?$AAc?$AAa?$AAt?$AAi@ 100023a8     esdhcbase_common_topaz_v1:esdhc.obj
 0001:00001418       ??_C@_1GI@COMJEFGB@?$AAC?$AAE?$AAS?$AAD?$AAH?$AAC?$AAB?$AAa?$AAs?$AAe?$AA?3?$AA?3?$AAI?$AAn?$AAi?$AAt?$AA?3?$AA?5?$AAE?$AAr?$AAr?$AAo?$AAr?$AA?5?$AAr?$AAe?$AAa?$AAd?$AAi?$AAn?$AAg?$AA?5@ 10002418     esdhcbase_common_topaz_v1:esdhc.obj
 0001:00001480       ??_C@_1HA@BOCMBEAP@?$AAC?$AAE?$AAS?$AAD?$AAH?$AAC?$AAB?$AAa?$AAs?$AAe?$AA?3?$AA?3?$AAI?$AAn?$AAi?$AAt?$AA?3?$AA?5?$AAF?$AAa?$AAi?$AAl?$AAe?$AAd?$AA?5?$AAt?$AAo?$AA?5?$AAa?$AAl?$AAl?$AAo@ 10002480     esdhcbase_common_topaz_v1:esdhc.obj
 0001:000014f0       ??_C@_1FM@JKMFPPEI@?$AAC?$AAE?$AAS?$AAD?$AAH?$AAC?$AAB?$AAa?$AAs?$AAe?$AA?3?$AA?3?$AAI?$AAn?$AAi?$AAt?$AA?3?$AA?5?$AAF?$AAa?$AAi?$AAl?$AAe?$AAd?$AA?5?$AAt?$AAo?$AA?5?$AAo?$AAp?$AAe?$AAn@ 100024f0     esdhcbase_common_topaz_v1:esdhc.obj
 0001:00001550       ??_C@_1FA@OLJGEDDE@?$AA?$CL?$AAC?$AAE?$AAS?$AAD?$AAH?$AAC?$AAB?$AAa?$AAs?$AAe?$AA?3?$AA?3?$AAI?$AAn?$AAi?$AAt?$AA?3?$AA?5?$AAA?$AAc?$AAt?$AAi?$AAv?$AAe?$AA?5?$AAR?$AAe?$AAg?$AAP?$AAa?$AAt@ 10002550     esdhcbase_common_topaz_v1:esdhc.obj
 0001:000015a0       ??_C@_1HI@LMNFJPNN@?$AAc?$AA?3?$AA?2?$AAw?$AAi?$AAn?$AAc?$AAe?$AAr?$AAo?$AAo?$AAt?$AAs?$AA?2?$AAt?$AAo?$AAp?$AAa?$AAz?$AA?2?$AAw?$AAi?$AAn?$AAc?$AAe?$AA7?$AA0?$AA0?$AA?2?$AAp?$AAu?$AAb@ 100025a0     esdhcbase_common_topaz_v1:esdhc.obj
 0001:00001618       ??_C@_1EE@PMALGIO@?$AA?9?$AAC?$AAE?$AAS?$AAD?$AAH?$AAC?$AAB?$AAa?$AAs?$AAe?$AA?3?$AA?3?$AAI?$AAO?$AAC?$AAo?$AAn?$AAt?$AAr?$AAo?$AAl?$AA?$CI?$AAr?$AAc?$AA?5?$AA?$DN?$AA?5?$AA?$CF?$AAd?$AA?$CJ?$AA?$AN@ 10002618     esdhcbase_common_topaz_v1:esdhc.obj
 0001:00001660       ??_C@_1GI@FHGICBHA@?$AAC?$AAE?$AAS?$AAD?$AAH?$AAC?$AAB?$AAa?$AAs?$AAe?$AA?3?$AA?3?$AAI?$AAO?$AAC?$AAo?$AAn?$AAt?$AAr?$AAo?$AAl?$AA?3?$AA?5?$AAU?$AAn?$AAk?$AAn?$AAo?$AAw?$AAn?$AA?5?$AAI@ 10002660     esdhcbase_common_topaz_v1:esdhc.obj
 0001:000016c8       ??_C@_1FK@IOCANBKN@?$AAC?$AAE?$AAS?$AAD?$AAH?$AAC?$AAB?$AAa?$AAs?$AAe?$AA?3?$AA?3?$AAI?$AAO?$AAC?$AAo?$AAn?$AAt?$AAr?$AAo?$AAl?$AA?3?$AA?5?$AAI?$AAO?$AAC?$AAT?$AAL?$AA_?$AAP?$AAO?$AAW@ 100026c8     esdhcbase_common_topaz_v1:esdhc.obj
 0001:00001728       ??_C@_1HI@PHKLBBMN@?$AAC?$AAE?$AAS?$AAD?$AAH?$AAC?$AAB?$AAa?$AAs?$AAe?$AA?3?$AA?3?$AAI?$AAO?$AAC?$AAo?$AAn?$AAt?$AAr?$AAo?$AAl?$AA?3?$AA?5?$AAI?$AAO?$AAC?$AAT?$AAL?$AA_?$AAP?$AAO?$AAW@ 10002728     esdhcbase_common_topaz_v1:esdhc.obj
 0001:000017a0       ??_C@_1IM@PCLBIGHL@?$AAC?$AAE?$AAS?$AAD?$AAH?$AAC?$AAB?$AAa?$AAs?$AAe?$AA?3?$AA?3?$AAI?$AAO?$AAC?$AAo?$AAn?$AAt?$AAr?$AAo?$AAl?$AA?3?$AA?5?$AAI?$AAO?$AAC?$AAT?$AAL?$AA_?$AAP?$AAO?$AAW@ 100027a0     esdhcbase_common_topaz_v1:esdhc.obj
 0001:00001830       ??_C@_1GC@GLMJMBMH@?$AAC?$AAE?$AAS?$AAD?$AAH?$AAC?$AAB?$AAa?$AAs?$AAe?$AA?3?$AA?3?$AAI?$AAO?$AAC?$AAo?$AAn?$AAt?$AAr?$AAo?$AAl?$AA?3?$AA?5?$AAC?$AAe?$AAS?$AAa?$AAf?$AAe?$AAC?$AAo?$AAp@ 10002830     esdhcbase_common_topaz_v1:esdhc.obj
 0001:00001898       ??_C@_1HC@GHHMKDML@?$AAC?$AAE?$AAS?$AAD?$AAH?$AAC?$AAB?$AAa?$AAs?$AAe?$AA?3?$AA?3?$AAI?$AAO?$AAC?$AAo?$AAn?$AAt?$AAr?$AAo?$AAl?$AA?3?$AA?5?$AAI?$AAO?$AAC?$AAT?$AAL?$AA_?$AAP?$AAO?$AAW@ 10002898     esdhcbase_common_topaz_v1:esdhc.obj
 0001:00001910       ??_C@_1IK@OOPDLKLH@?$AAC?$AAE?$AAS?$AAD?$AAH?$AAC?$AAB?$AAa?$AAs?$AAe?$AA?3?$AA?3?$AAI?$AAO?$AAC?$AAo?$AAn?$AAt?$AAr?$AAo?$AAl?$AA?3?$AA?5?$AAI?$AAO?$AAC?$AAT?$AAL?$AA_?$AAP?$AAO?$AAW@ 10002910     esdhcbase_common_topaz_v1:esdhc.obj
 0001:000019a0       ??_C@_1IC@MLLCDPOC@?$AA?$CL?$AAC?$AAE?$AAS?$AAD?$AAH?$AAC?$AAB?$AAa?$AAs?$AAe?$AA?3?$AA?3?$AAI?$AAO?$AAC?$AAo?$AAn?$AAt?$AAr?$AAo?$AAl?$AA?$CI?$AA0?$AAx?$AA?$CF?$AA0?$AA8?$AAx?$AA?0?$AA?5?$AA0@ 100029a0     esdhcbase_common_topaz_v1:esdhc.obj
 0001:00001a24       ??_C@_1M@LJLEHHPO@?$AAE?$AAS?$AAD?$AAH?$AAC?$AA?$AA@ 10002a24     esdhcbase_common_topaz_v1:esdhc.obj
 0001:00001a30       ??_C@_1IG@HNJLJDNI@?$AAC?$AAE?$AAS?$AAD?$AAH?$AAC?$AAB?$AAa?$AAs?$AAe?$AA?3?$AA?3?$AAS?$AAD?$AAH?$AAC?$AAI?$AAn?$AAi?$AAt?$AAi?$AAa?$AAl?$AAi?$AAz?$AAe?$AA?3?$AA?5?$AAE?$AAr?$AAr?$AAo@ 10002a30     esdhcbase_common_topaz_v1:esdhc.obj
 0001:00001ab8       ??_C@_1FG@GGFEFLAP@?$AAC?$AAE?$AAS?$AAD?$AAH?$AAC?$AAB?$AAa?$AAs?$AAe?$AA?3?$AA?3?$AAI?$AAn?$AAi?$AAt?$AA?3?$AA?5?$AAE?$AAr?$AAr?$AAo?$AAr?$AA?5?$AAw?$AAi?$AAt?$AAh?$AA?5?$AAI?$AAO?$AAM@ 10002ab8     esdhcbase_common_topaz_v1:esdhc.obj
 0001:00001b10       ??_C@_1FG@IBANJLHG@?$AAC?$AAE?$AAS?$AAD?$AAH?$AAC?$AAB?$AAa?$AAs?$AAe?$AA?3?$AA?3?$AAS?$AAt?$AAa?$AAr?$AAt?$AA?3?$AA?5?$AAP?$AAR?$AAO?$AAC?$AAT?$AAL?$AA?5?$AAs?$AAe?$AAt?$AA?5?$AAv?$AAa@ 10002b10     esdhcbase_common_topaz_v1:esdhc.obj
 0001:00001b68       ??_C@_1FI@PJKKJFIB@?$AAC?$AAE?$AAS?$AAD?$AAH?$AAC?$AAB?$AAa?$AAs?$AAe?$AAS?$AAD?$AAM?$AAA?$AA?3?$AAC?$AAr?$AAe?$AAa?$AAt?$AAe?$AA?5?$AAD?$AAM?$AAA?$AA?5?$AAO?$AAb?$AAj?$AAe?$AAc?$AAt@ 10002b68     esdhcbase_common_topaz_v1:esdhc.obj
 0001:00001bc0       ??_7CESDHCBaseSDMA@@6B@    10002bc0     esdhcbase_common_topaz_v1:esdhc.obj
 0001:00001be0       ??_C@_1FM@DIGHPNMF@?$AAS?$AAl?$AAo?$AAt?$AAp?$AAO?$AAp?$AAt?$AAi?$AAo?$AAn?$AAH?$AAa?$AAn?$AAd?$AAl?$AAe?$AAr?$AA?3?$AA?5?$AAC?$AAa?$AAp?$AAs?$AA?5?$AA?$DN?$AA?5?$AA0?$AAx?$AA?$CF?$AAx?$AA?0@ 10002be0     esdhcbase_common_topaz_v1:esdhc.obj
 0001:00001c40       ??_C@_1JO@CNNKFKDA@?$AAC?$AAE?$AAS?$AAD?$AAH?$AAC?$AAB?$AAa?$AAs?$AAe?$AA?3?$AA?3?$AAS?$AAD?$AAH?$AAC?$AAS?$AAl?$AAo?$AAt?$AAO?$AAp?$AAt?$AAi?$AAo?$AAn?$AAH?$AAa?$AAn?$AAd?$AAl?$AAe@ 10002c40     esdhcbase_common_topaz_v1:esdhc.obj
 0001:00001ce0       ??_C@_1JK@FEEDAAMF@?$AAC?$AAE?$AAS?$AAD?$AAH?$AAC?$AAB?$AAa?$AAs?$AAe?$AA?3?$AA?3?$AAS?$AAD?$AAH?$AAC?$AAS?$AAl?$AAo?$AAt?$AAO?$AAp?$AAt?$AAi?$AAo?$AAn?$AAH?$AAa?$AAn?$AAd?$AAl?$AAe@ 10002ce0     esdhcbase_common_topaz_v1:esdhc.obj
 0001:00001d80       ??_C@_1KO@NPEJPPCH@?$AAC?$AAE?$AAS?$AAD?$AAH?$AAC?$AAB?$AAa?$AAs?$AAe?$AA?3?$AA?3?$AAS?$AAD?$AAH?$AAC?$AAS?$AAl?$AAo?$AAt?$AAO?$AAp?$AAt?$AAi?$AAo?$AAn?$AAH?$AAa?$AAn?$AAd?$AAl?$AAe@ 10002d80     esdhcbase_common_topaz_v1:esdhc.obj
 0001:00001e30       ??_C@_1II@HDKCONND@?$AAC?$AAE?$AAS?$AAD?$AAH?$AAC?$AAB?$AAa?$AAs?$AAe?$AA?3?$AA?3?$AAS?$AAD?$AAH?$AAC?$AAS?$AAl?$AAo?$AAt?$AAO?$AAp?$AAt?$AAi?$AAo?$AAn?$AAH?$AAa?$AAn?$AAd?$AAl?$AAe@ 10002e30     esdhcbase_common_topaz_v1:esdhc.obj
 0001:00001eb8       ??_C@_1EG@FKLBFMGB@?$AA?9?$AAC?$AAE?$AAS?$AAD?$AAH?$AAC?$AAB?$AAa?$AAs?$AAe?$AA?3?$AA?3?$AAC?$AAo?$AAn?$AAt?$AAr?$AAo?$AAl?$AAl?$AAe?$AAr?$AAI?$AAs?$AAt?$AAT?$AAh?$AAr?$AAe?$AAa?$AAd@ 10002eb8     esdhcbase_common_topaz_v1:esdhc.obj
 0001:00001f00       ??_C@_1GG@OCJELOCK@?$AAC?$AAE?$AAS?$AAD?$AAH?$AAC?$AAB?$AAa?$AAs?$AAe?$AA?3?$AA?3?$AAC?$AAo?$AAn?$AAt?$AAr?$AAo?$AAl?$AAl?$AAe?$AAr?$AAI?$AAs?$AAt?$AAT?$AAh?$AAr?$AAe?$AAa?$AAd?$AA?3@ 10002f00     esdhcbase_common_topaz_v1:esdhc.obj
 0001:00001f68       ??_C@_1GA@MOHBMNLL@?$AAC?$AAE?$AAS?$AAD?$AAH?$AAC?$AAB?$AAa?$AAs?$AAe?$AA?3?$AA?3?$AAC?$AAo?$AAn?$AAt?$AAr?$AAo?$AAl?$AAl?$AAe?$AAr?$AAI?$AAs?$AAt?$AAT?$AAh?$AAr?$AAe?$AAa?$AAd?$AA?3@ 10002f68     esdhcbase_common_topaz_v1:esdhc.obj
 0001:00001fc8       ??_C@_1JG@ICLNBGPM@?$AAC?$AAE?$AAS?$AAD?$AAH?$AAC?$AAB?$AAa?$AAs?$AAe?$AA?3?$AA?3?$AAC?$AAo?$AAn?$AAt?$AAr?$AAo?$AAl?$AAl?$AAe?$AAr?$AAI?$AAs?$AAt?$AAT?$AAh?$AAr?$AAe?$AAa?$AAd?$AA?3@ 10002fc8     esdhcbase_common_topaz_v1:esdhc.obj
 0001:00002060       ??_C@_1IE@JLJFMAPE@?$AAC?$AAE?$AAS?$AAD?$AAH?$AAC?$AAB?$AAa?$AAs?$AAe?$AA?3?$AA?3?$AAS?$AAD?$AAH?$AAC?$AAB?$AAu?$AAs?$AAR?$AAe?$AAq?$AAu?$AAe?$AAs?$AAt?$AAH?$AAa?$AAn?$AAd?$AAl?$AAe@ 10003060     esdhcbase_common_topaz_v1:esdhc.obj
 0001:000020e8       ??_C@_1FO@CCGNBLBL@?$AAC?$AAE?$AAS?$AAD?$AAH?$AAC?$AAB?$AAa?$AAs?$AAe?$AA?3?$AA?3?$AAS?$AAD?$AAH?$AAC?$AAB?$AAu?$AAs?$AAR?$AAe?$AAq?$AAu?$AAe?$AAs?$AAt?$AAH?$AAa?$AAn?$AAd?$AAl?$AAe@ 100030e8     esdhcbase_common_topaz_v1:esdhc.obj
 0001:00002148       ??_C@_1IC@OPJNKLHC@?$AAC?$AAE?$AAS?$AAD?$AAH?$AAC?$AAB?$AAa?$AAs?$AAe?$AA?3?$AA?3?$AAG?$AAe?$AAt?$AAC?$AAo?$AAm?$AAm?$AAa?$AAn?$AAd?$AAR?$AAe?$AAs?$AAp?$AAo?$AAn?$AAs?$AAe?$AA?3?$AA?5@ 10003148     esdhcbase_common_topaz_v1:esdhc.obj
 0001:000021d0       ??_C@_1JE@EICBOPF@?$AAC?$AAE?$AAS?$AAD?$AAH?$AAC?$AAB?$AAa?$AAs?$AAe?$AA?3?$AA?3?$AAC?$AAo?$AAm?$AAm?$AAa?$AAn?$AAd?$AAC?$AAo?$AAm?$AAp?$AAl?$AAe?$AAt?$AAe?$AAH?$AAa?$AAn?$AAd?$AAl@ 100031d0     esdhcbase_common_topaz_v1:esdhc.obj
 0001:00002268       ??_C@_1EK@GMEKDPMA@?$AAC?$AAE?$AAS?$AAD?$AAH?$AAC?$AAB?$AAa?$AAs?$AAe?$AA?3?$AA?3?$AAC?$AAo?$AAm?$AAm?$AAa?$AAn?$AAd?$AAC?$AAo?$AAm?$AAp?$AAl?$AAe?$AAt?$AAe?$AAH?$AAa?$AAn?$AAd?$AAl@ 10003268     esdhcbase_common_topaz_v1:esdhc.obj
 0001:000022b8       ??_C@_1LM@BMOOHILM@?$AAC?$AAE?$AAS?$AAD?$AAH?$AAC?$AAB?$AAa?$AAs?$AAe?$AA?3?$AA?3?$AAI?$AAn?$AAd?$AAi?$AAc?$AAa?$AAt?$AAe?$AAB?$AAu?$AAs?$AAR?$AAe?$AAq?$AAu?$AAe?$AAs?$AAt?$AAC?$AAo@ 100032b8     esdhcbase_common_topaz_v1:esdhc.obj
 0001:00002378       ??_C@_1IK@JJPADEMK@?$AAC?$AAE?$AAS?$AAD?$AAH?$AAC?$AAB?$AAa?$AAs?$AAe?$AA?3?$AA?3?$AAI?$AAn?$AAd?$AAi?$AAc?$AAa?$AAt?$AAe?$AAB?$AAu?$AAs?$AAR?$AAe?$AAq?$AAu?$AAe?$AAs?$AAt?$AAC?$AAo@ 10003378     esdhcbase_common_topaz_v1:esdhc.obj
 0001:00002404       ??_C@_1CE@LNHBIFGC@?$AAS?$AAD?$AAH?$AAC?$AAI?$AAn?$AAi?$AAt?$AAi?$AAa?$AAl?$AAi?$AAz?$AAe?$AA?9?$AA?9?$AA?6?$AA?$AA@ 10003404     esdhcbase_common_topaz_v1:esdhc.obj
 0001:00002428       ??_C@_1CE@KNEHGPPI@?$AAS?$AAD?$AAH?$AAC?$AAI?$AAn?$AAi?$AAt?$AAi?$AAa?$AAl?$AAi?$AAz?$AAe?$AA?$CL?$AA?$CL?$AA?6?$AA?$AA@ 10003428     esdhcbase_common_topaz_v1:esdhc.obj
 0001:0000244c       ??_C@_1CI@KDNDCANC@?$AAS?$AAD?$AAH?$AAC?$AAD?$AAe?$AAi?$AAn?$AAi?$AAt?$AAi?$AAa?$AAl?$AAi?$AAz?$AAe?$AA?9?$AA?9?$AA?6?$AA?$AA@ 1000344c     esdhcbase_common_topaz_v1:esdhc.obj
 0001:00002474       ??_C@_1CI@LDOFMKEI@?$AAS?$AAD?$AAH?$AAC?$AAD?$AAe?$AAi?$AAn?$AAi?$AAt?$AAi?$AAa?$AAl?$AAi?$AAz?$AAe?$AA?$CL?$AA?$CL?$AA?6?$AA?$AA@ 10003474     esdhcbase_common_topaz_v1:esdhc.obj
 0001:0000249c       ??_7CESDHCBaseDMA@@6B@     1000349c     esdhcbase_common_topaz_v1:esdhcdma.obj
 0001:000024b8       ??_C@_1LA@MOACLCJN@?$AAc?$AA?3?$AA?2?$AAw?$AAi?$AAn?$AAc?$AAe?$AAr?$AAo?$AAo?$AAt?$AAs?$AA?2?$AAt?$AAo?$AAp?$AAa?$AAz?$AA?2?$AAw?$AAi?$AAn?$AAc?$AAe?$AA7?$AA0?$AA0?$AA?2?$AAp?$AAl?$AAa@ 100034b8     esdhcbase_common_topaz_v1:esdhcdma.obj
 0001:00002568       ??_C@_1GC@LIOJBPI@?$AAC?$AAE?$AAS?$AAD?$AAH?$AAC?$AAB?$AAa?$AAs?$AAe?$AA3?$AA2?$AAB?$AAi?$AAt?$AAA?$AAD?$AAM?$AAA?$AA?3?$AAC?$AAr?$AAe?$AAa?$AAt?$AAe?$AA?5?$AAD?$AAM?$AAA?$AA?5?$AAO@ 10003568     esdhcbase_common_topaz_v1:esdhcdma.obj
 0001:000025cc       ??_7CESDHCBase32BitADMA@@6B@ 100035cc     esdhcbase_common_topaz_v1:esdhcdma.obj
 0001:000025e8       ??_C@_1GG@EPFNGPKP@?$AAC?$AAE?$AAS?$AAD?$AAH?$AAC?$AAB?$AAa?$AAs?$AAe?$AA3?$AA2?$AAB?$AAi?$AAt?$AAA?$AAD?$AAM?$AAA?$AA2?$AA?3?$AAC?$AAr?$AAe?$AAa?$AAt?$AAe?$AA?5?$AAD?$AAM?$AAA?$AA?5@ 100035e8     esdhcbase_common_topaz_v1:esdhcdma.obj
 0001:00002650       ??_7CESDHCBase32BitADMA2@@6B@ 10003650     esdhcbase_common_topaz_v1:esdhcdma.obj
 0001:0000266c       ??_C@_1CO@PIELBKOM@?$AAA?$AAD?$AAM?$AAA?$AA?5?$AAE?$AAr?$AAr?$AAo?$AAr?$AA?5?$AAS?$AAt?$AAa?$AAt?$AAu?$AAs?$AA?5?$AA0?$AAx?$AA?$CF?$AAx?$AA?$AA@ 1000366c     esdhcbase_common_topaz_v1:esdhcdma.obj
 0001:0000269c       ??_C@_1DM@FNIHPPGH@?$AAS?$AAD?$AAC?$AAa?$AAr?$AAd?$AA?3?$AA?5?$AA?9?$AAS?$AAD?$AAI?$AAn?$AAi?$AAt?$AAi?$AAa?$AAl?$AAi?$AAz?$AAe?$AAC?$AAa?$AAr?$AAd?$AAL?$AAi?$AAb?$AA?6?$AA?$AA@ 1000369c     sdcardlib:SDMemApi.obj
 0001:000026d8       ??_C@_1IM@EHACHPD@?$AAd?$AA?3?$AA?2?$AAc?$AAh?$AAe?$AAl?$AAa?$AAn?$AAr?$AAt?$AAm?$AA2?$AA?2?$AAp?$AAu?$AAb?$AAl?$AAi?$AAc?$AA?2?$AAc?$AAo?$AAm?$AAm?$AAo?$AAn?$AA?2?$AAo?$AAa?$AAk?$AA?2@ 100036d8     sdcardlib:SDMemApi.obj
 0001:00002764       ??_C@_1DM@KBHHGOCL@?$AAS?$AAD?$AAC?$AAa?$AAr?$AAd?$AA?3?$AA?5?$AA?$CL?$AAS?$AAD?$AAI?$AAn?$AAi?$AAt?$AAi?$AAa?$AAl?$AAi?$AAz?$AAe?$AAC?$AAa?$AAr?$AAd?$AAL?$AAi?$AAb?$AA?6?$AA?$AA@ 10003764     sdcardlib:SDMemApi.obj
 0001:000027a0       ??_C@_1EA@IHEJNKEP@?$AAS?$AAD?$AAC?$AAa?$AAr?$AAd?$AA?3?$AA?5?$AA?9?$AAS?$AAD?$AAD?$AAe?$AAi?$AAn?$AAi?$AAt?$AAi?$AAa?$AAl?$AAi?$AAz?$AAe?$AAC?$AAa?$AAr?$AAd?$AAL?$AAi?$AAb?$AA?6?$AA?$AA@ 100037a0     sdcardlib:SDMemApi.obj
 0001:000027e0       ??_C@_1EA@KONLAIH@?$AAS?$AAD?$AAC?$AAa?$AAr?$AAd?$AA?3?$AA?5?$AA?$CL?$AAS?$AAD?$AAD?$AAe?$AAi?$AAn?$AAi?$AAt?$AAi?$AAa?$AAl?$AAi?$AAz?$AAe?$AAC?$AAa?$AAr?$AAd?$AAL?$AAi?$AAb?$AA?6?$AA?$AA@ 100037e0     sdcardlib:SDMemApi.obj
 0001:00002820       ??_C@_1EA@PKMJLCFO@?$AAS?$AAD?$AAC?$AAa?$AAr?$AAd?$AA?3?$AA?5?$AA?9?$AAA?$AAl?$AAl?$AAo?$AAc?$AAa?$AAt?$AAe?$AAM?$AAe?$AAm?$AAo?$AAr?$AAy?$AAW?$AAi?$AAt?$AAh?$AAT?$AAa?$AAg?$AA?6?$AA?$AA@ 10003820     sdcardlib:SDMemApi.obj
 0001:00002860       ??_C@_1EA@HHGNNIJG@?$AAS?$AAD?$AAC?$AAa?$AAr?$AAd?$AA?3?$AA?5?$AA?$CL?$AAA?$AAl?$AAl?$AAo?$AAc?$AAa?$AAt?$AAe?$AAM?$AAe?$AAm?$AAo?$AAr?$AAy?$AAW?$AAi?$AAt?$AAh?$AAT?$AAa?$AAg?$AA?6?$AA?$AA@ 10003860     sdcardlib:SDMemApi.obj
 0001:000028a0       ??_C@_1CO@CLLLMKPH@?$AAS?$AAD?$AAC?$AAa?$AAr?$AAd?$AA?3?$AA?5?$AA?9?$AAS?$AAD?$AAF?$AAr?$AAe?$AAe?$AAM?$AAe?$AAm?$AAo?$AAr?$AAy?$AA?6?$AA?$AA@ 100038a0     sdcardlib:SDMemApi.obj
 0001:000028d0       ??_C@_1CO@KCPJIAMH@?$AAS?$AAD?$AAC?$AAa?$AAr?$AAd?$AA?3?$AA?5?$AA?$CL?$AAS?$AAD?$AAF?$AAr?$AAe?$AAe?$AAM?$AAe?$AAm?$AAo?$AAr?$AAy?$AA?6?$AA?$AA@ 100038d0     sdcardlib:SDMemApi.obj
 0001:00002900       ??_C@_1DE@PNKBABJK@?$AAS?$AAD?$AAC?$AAa?$AAr?$AAd?$AA?3?$AA?5?$AA?9?$AAS?$AAD?$AAD?$AAe?$AAl?$AAe?$AAt?$AAe?$AAM?$AAe?$AAm?$AAL?$AAi?$AAs?$AAt?$AA?6?$AA?$AA@ 10003900     sdcardlib:SDMemApi.obj
 0001:00002938       ??_C@_1FI@EAJLBJMA@?$AAS?$AAD?$AAC?$AAa?$AAr?$AAd?$AA?3?$AA?5?$AAS?$AAD?$AAD?$AAe?$AAl?$AAe?$AAt?$AAe?$AAM?$AAe?$AAm?$AAL?$AAi?$AAs?$AAt?$AA?3?$AA?5?$AAI?$AAn?$AAv?$AAa?$AAl?$AAi?$AAd@ 10003938     sdcardlib:SDMemApi.obj
 0001:00002990       ??_C@_1DE@DEGBPGGG@?$AAS?$AAD?$AAC?$AAa?$AAr?$AAd?$AA?3?$AA?5?$AA?$CL?$AAS?$AAD?$AAD?$AAe?$AAl?$AAe?$AAt?$AAe?$AAM?$AAe?$AAm?$AAL?$AAi?$AAs?$AAt?$AA?6?$AA?$AA@ 10003990     sdcardlib:SDMemApi.obj
 0001:000029c4       ??_C@_1DK@IALNNOED@?$AAS?$AAD?$AAC?$AAa?$AAr?$AAd?$AA?3?$AA?5?$AA?9?$AAS?$AAD?$AAC?$AAr?$AAe?$AAa?$AAt?$AAe?$AAM?$AAe?$AAm?$AAo?$AAr?$AAy?$AAL?$AAi?$AAs?$AAt?$AA?6?$AA?$AA@ 100039c4     sdcardlib:SDMemApi.obj
 0001:00002a00       ??_C@_1HG@PLCNBJGG@?$AAS?$AAD?$AAC?$AAa?$AAr?$AAd?$AA?3?$AA?5?$AAS?$AAD?$AAC?$AAr?$AAe?$AAa?$AAt?$AAe?$AAM?$AAe?$AAm?$AAo?$AAr?$AAy?$AAL?$AAi?$AAs?$AAt?$AA?5?$AA?9?$AA?5?$AAF?$AAa?$AAi@ 10003a00     sdcardlib:SDMemApi.obj
 0001:00002a78       ??_C@_1JG@BHCAHMBD@?$AAS?$AAD?$AAC?$AAa?$AAr?$AAd?$AA?3?$AA?5?$AAW?$AAa?$AAr?$AAn?$AAi?$AAn?$AAg?$AA?3?$AA?5?$AAP?$AAl?$AAe?$AAa?$AAs?$AAe?$AA?5?$AAc?$AAa?$AAl?$AAl?$AA?5?$AAS?$AAD?$AAI@ 10003a78     sdcardlib:SDMemApi.obj
 0001:00002b10       ??_C@_1DK@PAMKMIKF@?$AAS?$AAD?$AAC?$AAa?$AAr?$AAd?$AA?3?$AA?5?$AA?$CL?$AAS?$AAD?$AAC?$AAr?$AAe?$AAa?$AAt?$AAe?$AAM?$AAe?$AAm?$AAo?$AAr?$AAy?$AAL?$AAi?$AAs?$AAt?$AA?6?$AA?$AA@ 10003b10     sdcardlib:SDMemApi.obj
 0001:00002b4c       ??_C@_1DE@PHIIFMNP@?$AAS?$AAD?$AAC?$AAa?$AAr?$AAd?$AA?3?$AA?5?$AA?9?$AAS?$AAD?$AAF?$AAr?$AAe?$AAe?$AAT?$AAo?$AAM?$AAe?$AAm?$AAL?$AAi?$AAs?$AAt?$AA?6?$AA?$AA@ 10003b4c     sdcardlib:SDMemApi.obj
 0001:00002b80       ??_C@_1FI@FMGJDFFO@?$AAS?$AAD?$AAC?$AAa?$AAr?$AAd?$AA?3?$AA?5?$AAS?$AAD?$AAF?$AAr?$AAe?$AAe?$AAT?$AAo?$AAM?$AAe?$AAm?$AAL?$AAi?$AAs?$AAt?$AA?3?$AA?5?$AAI?$AAn?$AAv?$AAa?$AAl?$AAi?$AAd@ 10003b80     sdcardlib:SDMemApi.obj
 0001:00002bd8       ??_C@_1DE@DOEIKLCD@?$AAS?$AAD?$AAC?$AAa?$AAr?$AAd?$AA?3?$AA?5?$AA?$CL?$AAS?$AAD?$AAF?$AAr?$AAe?$AAe?$AAT?$AAo?$AAM?$AAe?$AAm?$AAL?$AAi?$AAs?$AAt?$AA?6?$AA?$AA@ 10003bd8     sdcardlib:SDMemApi.obj
 0001:00002c10       ??_C@_1EA@MGFGENGM@?$AAS?$AAD?$AAC?$AAa?$AAr?$AAd?$AA?3?$AA?5?$AA?9?$AAS?$AAD?$AAA?$AAl?$AAl?$AAo?$AAc?$AAa?$AAt?$AAe?$AAF?$AAr?$AAo?$AAm?$AAM?$AAe?$AAm?$AAL?$AAi?$AAs?$AAt?$AA?6?$AA?$AA@ 10003c10     sdcardlib:SDMemApi.obj
 0001:00002c50       ??_C@_1GE@ECPANGPG@?$AAS?$AAD?$AAC?$AAa?$AAr?$AAd?$AA?3?$AA?5?$AAS?$AAD?$AAA?$AAl?$AAl?$AAo?$AAc?$AAa?$AAt?$AAe?$AAF?$AAr?$AAo?$AAm?$AAM?$AAe?$AAm?$AAL?$AAi?$AAs?$AAt?$AA?3?$AA?5?$AAI@ 10003c50     sdcardlib:SDMemApi.obj
 0001:00002cb8       ??_C@_1EA@ELPCCHKE@?$AAS?$AAD?$AAC?$AAa?$AAr?$AAd?$AA?3?$AA?5?$AA?$CL?$AAS?$AAD?$AAA?$AAl?$AAl?$AAo?$AAc?$AAa?$AAt?$AAe?$AAF?$AAr?$AAo?$AAm?$AAM?$AAe?$AAm?$AAL?$AAi?$AAs?$AAt?$AA?6?$AA?$AA@ 10003cb8     sdcardlib:SDMemApi.obj
 0001:00002cf8       ??_C@_1HA@CHFKMAIE@?$AAd?$AA?3?$AA?2?$AAc?$AAh?$AAe?$AAl?$AAa?$AAn?$AAr?$AAt?$AAm?$AA2?$AA?2?$AAp?$AAu?$AAb?$AAl?$AAi?$AAc?$AA?2?$AAc?$AAo?$AAm?$AAm?$AAo?$AAn?$AA?2?$AAs?$AAd?$AAk?$AA?2@ 10003cf8     sdcardlib:SDMemApi.obj
 0001:00002d68       ??_C@_1IK@MFJACAMD@?$AAd?$AA?3?$AA?2?$AAc?$AAh?$AAe?$AAl?$AAa?$AAn?$AAr?$AAt?$AAm?$AA2?$AA?2?$AAp?$AAu?$AAb?$AAl?$AAi?$AAc?$AA?2?$AAc?$AAo?$AAm?$AAm?$AAo?$AAn?$AA?2?$AAo?$AAa?$AAk?$AA?2@ 10003d68     sdcardlib:SDDebug.obj
 0001:00002df8       ??_C@_1II@GMHCLLNI@?$AA?5?$AAE?$AAX?$AAC?$AAE?$AAP?$AAT?$AAI?$AAO?$AAN?$AA_?$AAA?$AAC?$AAC?$AAE?$AAS?$AAS?$AA_?$AAV?$AAI?$AAO?$AAL?$AAA?$AAT?$AAI?$AAO?$AAN?$AA?5?$AAr?$AAa?$AAi?$AAs@ 10003df8     sdcardlib:SDDebug.obj
 0001:00002e80       ??_C@_1HA@BGPDKPFE@?$AA?5?$AA?5?$AA?5?$AA?5?$AA?5?$AA?5?$AA?5?$AA?5?$AAW?$AAr?$AAi?$AAt?$AAe?$AA?5?$AAA?$AAc?$AAc?$AAe?$AAs?$AAs?$AA?5?$AAE?$AAx?$AAc?$AAe?$AAp?$AAt?$AAi?$AAo?$AAn?$AAe?$AAd@ 10003e80     sdcardlib:SDDebug.obj
 0001:00002ef0       ??_C@_1GO@LIPPKMGO@?$AA?5?$AA?5?$AA?5?$AA?5?$AA?5?$AA?5?$AA?5?$AA?5?$AAR?$AAe?$AAa?$AAd?$AA?5?$AAA?$AAc?$AAc?$AAe?$AAs?$AAs?$AA?5?$AAE?$AAx?$AAc?$AAe?$AAp?$AAt?$AAi?$AAo?$AAn?$AAe?$AAd?$AA?5@ 10003ef0     sdcardlib:SDDebug.obj
 0001:00002f60       ??_C@_1DK@CNMPAAFJ@?$AA?5?$AA?5?$AA?5?$AA?5?$AA?5?$AA?5?$AA?5?$AA?5?$AAE?$AAx?$AAc?$AAe?$AAp?$AAt?$AAi?$AAo?$AAn?$AA?3?$AA?5?$AAU?$AAN?$AAK?$AAN?$AAO?$AAW?$AAN?$AA?5?$AA?6?$AA?$AA@ 10003f60     sdcardlib:SDDebug.obj
 0001:00002fa0       ??_C@_1FM@BABDDJHM@?$AA?5?$AA?5?$AA?5?$AA?5?$AA?5?$AA?5?$AA?5?$AA?5?$AAE?$AAx?$AAc?$AAe?$AAp?$AAt?$AAi?$AAo?$AAn?$AA?3?$AA?5?$AAE?$AAX?$AAC?$AAE?$AAP?$AAT?$AAI?$AAO?$AAN?$AA_?$AAI?$AAN?$AAV@ 10003fa0     sdcardlib:SDDebug.obj
 0001:00003000       ??_C@_1FE@FKGKNFOP@?$AA?5?$AA?5?$AA?5?$AA?5?$AA?5?$AA?5?$AA?5?$AA?5?$AAE?$AAx?$AAc?$AAe?$AAp?$AAt?$AAi?$AAo?$AAn?$AA?3?$AA?5?$AAE?$AAX?$AAC?$AAE?$AAP?$AAT?$AAI?$AAO?$AAN?$AA_?$AAG?$AAU?$AAA@ 10004000     sdcardlib:SDDebug.obj
 0001:00003058       ??_C@_1GG@EOOLNNB@?$AA?5?$AA?5?$AA?5?$AA?5?$AA?5?$AA?5?$AA?5?$AA?5?$AAE?$AAx?$AAc?$AAe?$AAp?$AAt?$AAi?$AAo?$AAn?$AA?3?$AA?5?$AAE?$AAX?$AAC?$AAE?$AAP?$AAT?$AAI?$AAO?$AAN?$AA_?$AAI?$AAN?$AAV@ 10004058     sdcardlib:SDDebug.obj
 0001:000030c0       ??_C@_1FM@DAEFKFAP@?$AA?5?$AA?5?$AA?5?$AA?5?$AA?5?$AA?5?$AA?5?$AA?5?$AAE?$AAx?$AAc?$AAe?$AAp?$AAt?$AAi?$AAo?$AAn?$AA?3?$AA?5?$AAE?$AAX?$AAC?$AAE?$AAP?$AAT?$AAI?$AAO?$AAN?$AA_?$AAS?$AAT?$AAA@ 100040c0     sdcardlib:SDDebug.obj
 0001:00003120       ??_C@_1HA@NODJFEFD@?$AA?5?$AA?5?$AA?5?$AA?5?$AA?5?$AA?5?$AA?5?$AA?5?$AAE?$AAx?$AAc?$AAe?$AAp?$AAt?$AAi?$AAo?$AAn?$AA?3?$AA?5?$AAE?$AAX?$AAC?$AAE?$AAP?$AAT?$AAI?$AAO?$AAN?$AA_?$AAN?$AAO?$AAN@ 10004120     sdcardlib:SDDebug.obj
 0001:00003190       ??_C@_1GG@OHPADMDK@?$AA?5?$AA?5?$AA?5?$AA?5?$AA?5?$AA?5?$AA?5?$AA?5?$AAE?$AAx?$AAc?$AAe?$AAp?$AAt?$AAi?$AAo?$AAn?$AA?3?$AA?5?$AAE?$AAX?$AAC?$AAE?$AAP?$AAT?$AAI?$AAO?$AAN?$AA_?$AAI?$AAL?$AAL@ 10004190     sdcardlib:SDDebug.obj
 0001:000031f8       ??_C@_1FK@HMKLGOCN@?$AA?5?$AA?5?$AA?5?$AA?5?$AA?5?$AA?5?$AA?5?$AA?5?$AAE?$AAx?$AAc?$AAe?$AAp?$AAt?$AAi?$AAo?$AAn?$AA?3?$AA?5?$AAE?$AAX?$AAC?$AAE?$AAP?$AAT?$AAI?$AAO?$AAN?$AA_?$AAI?$AAN?$AA_@ 100041f8     sdcardlib:SDDebug.obj
 0001:00003258       ??_C@_1GA@IHGOLIHL@?$AA?5?$AA?5?$AA?5?$AA?5?$AA?5?$AA?5?$AA?5?$AA?5?$AAE?$AAx?$AAc?$AAe?$AAp?$AAt?$AAi?$AAo?$AAn?$AA?3?$AA?5?$AAE?$AAX?$AAC?$AAE?$AAP?$AAT?$AAI?$AAO?$AAN?$AA_?$AAP?$AAR?$AAI@ 10004258     sdcardlib:SDDebug.obj
 0001:000032b8       ??_C@_1FI@BCFEANND@?$AA?5?$AA?5?$AA?5?$AA?5?$AA?5?$AA?5?$AA?5?$AA?5?$AAE?$AAx?$AAc?$AAe?$AAp?$AAt?$AAi?$AAo?$AAn?$AA?3?$AA?5?$AAE?$AAX?$AAC?$AAE?$AAP?$AAT?$AAI?$AAO?$AAN?$AA_?$AAI?$AAN?$AAT@ 100042b8     sdcardlib:SDDebug.obj
 0001:00003310       ??_C@_1GE@PJCCPNIC@?$AA?5?$AA?5?$AA?5?$AA?5?$AA?5?$AA?5?$AA?5?$AA?5?$AAE?$AAx?$AAc?$AAe?$AAp?$AAt?$AAi?$AAo?$AAn?$AA?3?$AA?5?$AAE?$AAX?$AAC?$AAE?$AAP?$AAT?$AAI?$AAO?$AAN?$AA_?$AAI?$AAN?$AAT@ 10004310     sdcardlib:SDDebug.obj
 0001:00003378       ??_C@_1FK@PFDOHDMA@?$AA?5?$AA?5?$AA?5?$AA?5?$AA?5?$AA?5?$AA?5?$AA?5?$AAE?$AAx?$AAc?$AAe?$AAp?$AAt?$AAi?$AAo?$AAn?$AA?3?$AA?5?$AAE?$AAX?$AAC?$AAE?$AAP?$AAT?$AAI?$AAO?$AAN?$AA_?$AAF?$AAL?$AAT@ 10004378     sdcardlib:SDDebug.obj
 0001:000033d8       ??_C@_1FO@KLJPJDBD@?$AA?5?$AA?5?$AA?5?$AA?5?$AA?5?$AA?5?$AA?5?$AA?5?$AAE?$AAx?$AAc?$AAe?$AAp?$AAt?$AAi?$AAo?$AAn?$AA?3?$AA?5?$AAE?$AAX?$AAC?$AAE?$AAP?$AAT?$AAI?$AAO?$AAN?$AA_?$AAF?$AAL?$AAT@ 100043d8     sdcardlib:SDDebug.obj
 0001:00003438       ??_C@_1FI@JMGLEANA@?$AA?5?$AA?5?$AA?5?$AA?5?$AA?5?$AA?5?$AA?5?$AA?5?$AAE?$AAx?$AAc?$AAe?$AAp?$AAt?$AAi?$AAo?$AAn?$AA?3?$AA?5?$AAE?$AAX?$AAC?$AAE?$AAP?$AAT?$AAI?$AAO?$AAN?$AA_?$AAF?$AAL?$AAT@ 10004438     sdcardlib:SDDebug.obj
 0001:00003490       ??_C@_1GK@PFCJLJFD@?$AA?5?$AA?5?$AA?5?$AA?5?$AA?5?$AA?5?$AA?5?$AA?5?$AAE?$AAx?$AAc?$AAe?$AAp?$AAt?$AAi?$AAo?$AAn?$AA?3?$AA?5?$AAE?$AAX?$AAC?$AAE?$AAP?$AAT?$AAI?$AAO?$AAN?$AA_?$AAF?$AAL?$AAT@ 10004490     sdcardlib:SDDebug.obj
 0001:00003500       ??_C@_1GE@IFHGPJDI@?$AA?5?$AA?5?$AA?5?$AA?5?$AA?5?$AA?5?$AA?5?$AA?5?$AAE?$AAx?$AAc?$AAe?$AAp?$AAt?$AAi?$AAo?$AAn?$AA?3?$AA?5?$AAE?$AAX?$AAC?$AAE?$AAP?$AAT?$AAI?$AAO?$AAN?$AA_?$AAF?$AAL?$AAT@ 10004500     sdcardlib:SDDebug.obj
 0001:00003568       ??_C@_1GE@KEAPHJPC@?$AA?5?$AA?5?$AA?5?$AA?5?$AA?5?$AA?5?$AA?5?$AA?5?$AAE?$AAx?$AAc?$AAe?$AAp?$AAt?$AAi?$AAo?$AAn?$AA?3?$AA?5?$AAE?$AAX?$AAC?$AAE?$AAP?$AAT?$AAI?$AAO?$AAN?$AA_?$AAF?$AAL?$AAT@ 10004568     sdcardlib:SDDebug.obj
 0001:000035d0       ??_C@_1GI@FODJCDCC@?$AA?5?$AA?5?$AA?5?$AA?5?$AA?5?$AA?5?$AA?5?$AA?5?$AAE?$AAx?$AAc?$AAe?$AAp?$AAt?$AAi?$AAo?$AAn?$AA?3?$AA?5?$AAE?$AAX?$AAC?$AAE?$AAP?$AAT?$AAI?$AAO?$AAN?$AA_?$AAF?$AAL?$AAT@ 100045d0     sdcardlib:SDDebug.obj
 0001:00003638       ??_C@_1GK@BIDJEADM@?$AA?5?$AA?5?$AA?5?$AA?5?$AA?5?$AA?5?$AA?5?$AA?5?$AAE?$AAx?$AAc?$AAe?$AAp?$AAt?$AAi?$AAo?$AAn?$AA?3?$AA?5?$AAE?$AAX?$AAC?$AAE?$AAP?$AAT?$AAI?$AAO?$AAN?$AA_?$AAA?$AAR?$AAR@ 10004638     sdcardlib:SDDebug.obj
 0001:000036a8       ??_C@_1FG@FAMEFIJC@?$AA?5?$AA?5?$AA?5?$AA?5?$AA?5?$AA?5?$AA?5?$AA?5?$AAE?$AAx?$AAc?$AAe?$AAp?$AAt?$AAi?$AAo?$AAn?$AA?3?$AA?5?$AAE?$AAX?$AAC?$AAE?$AAP?$AAT?$AAI?$AAO?$AAN?$AA_?$AAS?$AAI?$AAN@ 100046a8     sdcardlib:SDDebug.obj
 0001:00003700       ??_C@_1FE@LHIOIAHH@?$AA?5?$AA?5?$AA?5?$AA?5?$AA?5?$AA?5?$AA?5?$AA?5?$AAE?$AAx?$AAc?$AAe?$AAp?$AAt?$AAi?$AAo?$AAn?$AA?3?$AA?5?$AAE?$AAX?$AAC?$AAE?$AAP?$AAT?$AAI?$AAO?$AAN?$AA_?$AAB?$AAR?$AAE@ 10004700     sdcardlib:SDDebug.obj
 0001:00003758       ??_C@_1GK@NIJAGIMI@?$AA?5?$AA?5?$AA?5?$AA?5?$AA?5?$AA?5?$AA?5?$AA?5?$AAE?$AAx?$AAc?$AAe?$AAp?$AAt?$AAi?$AAo?$AAn?$AA?3?$AA?5?$AAE?$AAX?$AAC?$AAE?$AAP?$AAT?$AAI?$AAO?$AAN?$AA_?$AAD?$AAA?$AAT@ 10004758     sdcardlib:SDDebug.obj
 0001:000037c8       ??_C@_1GA@IMOMELNN@?$AA?5?$AA?5?$AA?5?$AA?5?$AA?5?$AA?5?$AA?5?$AA?5?$AAE?$AAx?$AAc?$AAe?$AAp?$AAt?$AAi?$AAo?$AAn?$AA?3?$AA?5?$AAE?$AAX?$AAC?$AAE?$AAP?$AAT?$AAI?$AAO?$AAN?$AA_?$AAA?$AAC?$AAC@ 100047c8     sdcardlib:SDDebug.obj
 0001:00003828       ??_C@_1LA@GNONOPLI@?$AAS?$AAD?$AAB?$AAu?$AAs?$AAD?$AAr?$AAi?$AAv?$AAe?$AAr?$AA?3?$AA?5?$AAE?$AAx?$AAc?$AAe?$AAp?$AAt?$AAi?$AAo?$AAn?$AA?5?$AAc?$AAa?$AAu?$AAg?$AAh?$AAt?$AA?5?$AAE?$AAx@ 10004828     sdcardlib:SDDebug.obj
 0001:000038d8       ??_C@_1JI@EFCALCGP@?$AAS?$AAD?$AAP?$AAe?$AAr?$AAf?$AAo?$AAr?$AAm?$AAS?$AAa?$AAf?$AAe?$AAC?$AAo?$AAp?$AAy?$AA?5?$AA?$CI?$AAD?$AAe?$AAs?$AAt?$AA?3?$AA?5?$AA0?$AAx?$AA?$CF?$AA0?$AA8?$AAX?$AA?$CJ@ 100048d8     sdcardlib:SDDebug.obj
 0001:00003970       ??_C@_1EO@NDAHAEDP@?$AAS?$AAD?$AAC?$AAa?$AAr?$AAd?$AAL?$AAi?$AAb?$AA?3?$AA?5?$AAE?$AAx?$AAc?$AAe?$AAp?$AAt?$AAi?$AAo?$AAn?$AA?5?$AAi?$AAn?$AA?5?$AAS?$AAD?$AAO?$AAu?$AAt?$AAp?$AAu?$AAB@ 10004970     sdcardlib:SDDebug.obj
 0001:000039c0       ??_C@_17MJEANDKP@?$AA?$CF?$AAs?$AA?6?$AA?$AA@ 100049c0     sdcardlib:SDDebug.obj
 0001:000039c8       ??_C@_17MEDFOIMI@?$AA?5?$AA?5?$AA?5?$AA?$AA@ 100049c8     sdcardlib:SDDebug.obj
 0001:000039d0       ??_C@_1M@OLEMGGOE@?$AA?$CF?$AA0?$AA2?$AAX?$AA?5?$AA?$AA@ 100049d0     sdcardlib:SDDebug.obj
 0001:000039dc       ??_C@_1BE@DCNBFMAB@?$AA?5?$AA0?$AAx?$AA?$CF?$AA0?$AA8?$AAX?$AA?5?$AA?5?$AA?$AA@ 100049dc     sdcardlib:SDDebug.obj
 0001:000039f0       ??_C@_1FC@CNHMKNPP@?$AAS?$AAD?$AAO?$AAu?$AAt?$AAp?$AAu?$AAt?$AAB?$AAu?$AAf?$AAf?$AAe?$AAr?$AA?3?$AA?5?$AA0?$AAx?$AA?$CF?$AA0?$AA8?$AAX?$AA?5?$AA?0?$AA?5?$AAS?$AAi?$AAz?$AAe?$AA?3?$AA?5?$AA?$CF@ 100049f0     sdcardlib:SDDebug.obj
 0001:00003a48       ??_C@_1LE@CEKDGLLA@?$AA?9?$AA?9?$AA?9?$AA?9?$AA?9?$AA?9?$AA?9?$AA?9?$AA?9?$AA?9?$AA?9?$AA?9?$AA?9?$AA?9?$AA?9?$AA?9?$AA?9?$AA?9?$AA?9?$AA?9?$AA?9?$AA?9?$AA?9?$AA?9?$AA?9?$AA?9?$AA?9?$AA?9?$AA?9?$AA?9?$AA?9?$AA?9@ 10004a48     sdcardlib:SDDebug.obj
 0001:00003b00       ??_C@_1GE@HBHOBMJ@?$AAS?$AAD?$AAR?$AAe?$AAg?$AAi?$AAs?$AAt?$AAe?$AAr?$AAC?$AAl?$AAi?$AAe?$AAn?$AAt?$AA?3?$AA?5?$AAF?$AAa?$AAi?$AAl?$AAe?$AAd?$AA?5?$AAt?$AAo?$AA?5?$AAg?$AAe?$AAt?$AA?5@ 10004b00     sdcardlib:SDCardApiStubs.obj
 0001:00003b68       ??_C@_1JI@JGAJMFAG@?$AAd?$AA?3?$AA?2?$AAc?$AAh?$AAe?$AAl?$AAa?$AAn?$AAr?$AAt?$AAm?$AA2?$AA?2?$AAp?$AAu?$AAb?$AAl?$AAi?$AAc?$AA?2?$AAc?$AAo?$AAm?$AAm?$AAo?$AAn?$AA?2?$AAo?$AAa?$AAk?$AA?2@ 10004b68     sdcardlib:SDCardApiStubs.obj
 0001:00003c00       ??_C@_1HE@HJICDLFD@?$AAd?$AA?3?$AA?2?$AAc?$AAh?$AAe?$AAl?$AAa?$AAn?$AAr?$AAt?$AAm?$AA2?$AA?2?$AAp?$AAr?$AAi?$AAv?$AAa?$AAt?$AAe?$AA?2?$AAw?$AAi?$AAn?$AAc?$AAe?$AAo?$AAs?$AA?2?$AAc?$AAo@ 10004c00     sdcardlib:utilmem.obj
 0001:00003c78       ??_C@_1HG@PCOMHGCB@?$AAd?$AA?3?$AA?2?$AAc?$AAh?$AAe?$AAl?$AAa?$AAn?$AAr?$AAt?$AAm?$AA2?$AA?2?$AAp?$AAr?$AAi?$AAv?$AAa?$AAt?$AAe?$AA?2?$AAw?$AAi?$AAn?$AAc?$AAe?$AAo?$AAs?$AA?2?$AAc?$AAo@ 10004c78     sdcardlib:utilmemf.obj
 0001:00003cf0       ??_C@_1GA@HFJEPHCP@?$AAd?$AA?3?$AA?2?$AAc?$AAh?$AAe?$AAl?$AAa?$AAn?$AAr?$AAt?$AAm?$AA2?$AA?2?$AAp?$AAu?$AAb?$AAl?$AAi?$AAc?$AA?2?$AAc?$AAo?$AAm?$AAm?$AAo?$AAn?$AA?2?$AAs?$AAd?$AAk?$AA?2@ 10004cf0     sdcardlib:utilmemf.obj
 0001:00003d50       ??_7SVSTree@@6B@           10004d50     sdcardlib:utilmemf.obj
 0001:00003d60       ??_7SVSEnumClass@@6B@      10004d60     sdcardlib:utilmemf.obj
 0001:00003d70       ??_C@_1HI@GJBOOHGA@?$AAB?$AAu?$AAs?$AAI?$AAo?$AA?5?$AAf?$AAo?$AAr?$AA?5?$AAS?$AAD?$AAR?$AAe?$AAg?$AAi?$AAs?$AAt?$AAe?$AAr?$AAC?$AAl?$AAi?$AAe?$AAn?$AAt?$AA_?$AA_?$AAX?$AA?3?$AA?5?$AAF@ 10004d70     sdcardlib:busacc.obj
 0001:00003de8       ??_C@_1IG@KNCDAMMP@?$AAB?$AAu?$AAs?$AAI?$AAo?$AA?5?$AAf?$AAo?$AAr?$AA?5?$AAS?$AAD?$AAS?$AAy?$AAn?$AAc?$AAh?$AAr?$AAo?$AAn?$AAo?$AAu?$AAs?$AAB?$AAu?$AAs?$AAR?$AAe?$AAq?$AAu?$AAe?$AAs@ 10004de8     sdcardlib:busacc.obj
 0001:00003e70       ??_C@_1GM@PAOFIFOM@?$AAS?$AAD?$AAB?$AAu?$AAs?$AAR?$AAe?$AAq?$AAu?$AAe?$AAs?$AAt?$AAR?$AAe?$AAs?$AAp?$AAo?$AAn?$AAs?$AAe?$AA_?$AA_?$AAX?$AA?3?$AA?5?$AAF?$AAa?$AAi?$AAl?$AAe?$AAd?$AA?3@ 10004e70     sdcardlib:busacc.obj
 0001:00003ee0       ??_C@_1IA@CIBMOFCE@?$AAB?$AAu?$AAs?$AAI?$AAo?$AA?5?$AAf?$AAo?$AAr?$AA?5?$AAS?$AAD?$AAB?$AAu?$AAs?$AAR?$AAe?$AAq?$AAu?$AAe?$AAs?$AAt?$AAR?$AAe?$AAs?$AAp?$AAo?$AAn?$AAs?$AAe?$AA_?$AA_@ 10004ee0     sdcardlib:busacc.obj
 0001:00003f60       ??_C@_1HA@IJKGFFPM@?$AAB?$AAu?$AAs?$AAI?$AAo?$AA?5?$AAf?$AAo?$AAr?$AA?5?$AAS?$AAD?$AAB?$AAu?$AAs?$AAR?$AAe?$AAq?$AAu?$AAe?$AAs?$AAt?$AA_?$AA_?$AAX?$AA?3?$AA?5?$AAF?$AAa?$AAi?$AAl?$AAe@ 10004f60     sdcardlib:busacc.obj
 0001:00003fd0       ??_C@_1HM@HHAOJEME@?$AAB?$AAu?$AAs?$AAI?$AAo?$AA?5?$AAf?$AAo?$AAr?$AA?5?$AAS?$AAD?$AAC?$AAa?$AAn?$AAc?$AAe?$AAl?$AAB?$AAu?$AAs?$AAR?$AAe?$AAq?$AAu?$AAe?$AAs?$AAt?$AA_?$AA_?$AAX?$AA?3@ 10004fd0     sdcardlib:busacc.obj
 0001:00004050       ??_C@_1HI@OPHKAJHO@?$AAB?$AAu?$AAs?$AAI?$AAo?$AA?5?$AAf?$AAo?$AAr?$AA?5?$AAS?$AAD?$AAF?$AAr?$AAe?$AAe?$AAB?$AAu?$AAs?$AAR?$AAe?$AAq?$AAu?$AAe?$AAs?$AAt?$AA_?$AA_?$AAX?$AA?3?$AA?5?$AAF@ 10005050     sdcardlib:busacc.obj
 0001:000040c8       ??_C@_1HG@PFEJGILM@?$AAB?$AAu?$AAs?$AAI?$AAo?$AA?5?$AAf?$AAo?$AAr?$AA?5?$AAS?$AAD?$AAC?$AAa?$AAr?$AAd?$AAI?$AAn?$AAf?$AAo?$AAQ?$AAu?$AAe?$AAr?$AAy?$AA_?$AA_?$AAX?$AA?3?$AA?5?$AAF?$AAa@ 100050c8     sdcardlib:busacc.obj
 0001:00004140       ??_C@_1IM@NOMNMOBB@?$AAB?$AAu?$AAs?$AAI?$AAo?$AA?5?$AAf?$AAo?$AAr?$AA?5?$AAS?$AAD?$AAR?$AAe?$AAa?$AAd?$AAW?$AAr?$AAi?$AAt?$AAe?$AAR?$AAe?$AAg?$AAi?$AAs?$AAt?$AAe?$AAr?$AAs?$AAD?$AAi@ 10005140     sdcardlib:busacc.obj
 0001:000041d0       ??_C@_1IA@CLANCPLA@?$AAB?$AAu?$AAs?$AAI?$AAo?$AA?5?$AAf?$AAo?$AAr?$AA?5?$AAS?$AAD?$AAI?$AAO?$AAC?$AAo?$AAn?$AAn?$AAe?$AAc?$AAt?$AAI?$AAn?$AAt?$AAe?$AAr?$AAr?$AAu?$AAp?$AAt?$AA_?$AA_@ 100051d0     sdcardlib:busacc.obj
 0001:00004250       ??_C@_1IG@IHCPJIGO@?$AAB?$AAu?$AAs?$AAI?$AAo?$AA?5?$AAf?$AAo?$AAr?$AA?5?$AAS?$AAD?$AAI?$AAO?$AAD?$AAi?$AAs?$AAc?$AAo?$AAn?$AAn?$AAe?$AAc?$AAt?$AAI?$AAn?$AAt?$AAe?$AAr?$AAr?$AAu?$AAp@ 10005250     sdcardlib:busacc.obj
 0001:000042d8       ??_C@_1HI@DDPJLEDO@?$AAB?$AAu?$AAs?$AAI?$AAo?$AA?5?$AAf?$AAo?$AAr?$AA?5?$AAS?$AAD?$AAS?$AAe?$AAt?$AAC?$AAa?$AAr?$AAd?$AAF?$AAe?$AAa?$AAt?$AAu?$AAr?$AAe?$AA_?$AA_?$AAX?$AA?3?$AA?5?$AAF@ 100052d8     sdcardlib:busacc.obj
 0001:00004350       ??_C@_1DK@DAPDOICG@?$AAA?$AAs?$AAs?$AAe?$AAr?$AAt?$AA?5?$AAb?$AAr?$AAo?$AAk?$AAe?$AAn?$AA?5?$AAi?$AAn?$AA?5?$AA?$CF?$AAs?$AA?5?$AAl?$AAi?$AAn?$AAe?$AA?5?$AA?$CF?$AAd?$AA?6?$AA?$AA@ 10005350     sdcardlib:svsutil.obj
 0001:00004390       ??_C@_1HG@HLFFDIPJ@?$AAd?$AA?3?$AA?2?$AAc?$AAh?$AAe?$AAl?$AAa?$AAn?$AAr?$AAt?$AAm?$AA2?$AA?2?$AAp?$AAr?$AAi?$AAv?$AAa?$AAt?$AAe?$AA?2?$AAw?$AAi?$AAn?$AAc?$AAe?$AAo?$AAs?$AA?2?$AAc?$AAo@ 10005390     sdcardlib:utiltree.obj
 0001:00004408       ??_C@_1GE@JPPCAFMN@?$AAS?$AAD?$AAH?$AAC?$AAD?$AAI?$AAn?$AAi?$AAt?$AAi?$AAa?$AAl?$AAi?$AAz?$AAe?$AAH?$AAC?$AAL?$AAi?$AAb?$AA?3?$AA?5?$AAF?$AAa?$AAi?$AAl?$AAe?$AAd?$AA?5?$AAt?$AAo?$AA?5@ 10005408     sdhclib:SDHCLib.obj
 0001:00004470       ??_C@_1IG@CLDCKGMJ@?$AAd?$AA?3?$AA?2?$AAc?$AAh?$AAe?$AAl?$AAa?$AAn?$AAr?$AAt?$AAm?$AA2?$AA?2?$AAp?$AAu?$AAb?$AAl?$AAi?$AAc?$AA?2?$AAc?$AAo?$AAm?$AAm?$AAo?$AAn?$AA?2?$AAo?$AAa?$AAk?$AA?2@ 10005470     sdhclib:SDHCLib.obj
 0001:0000451c       ?BspGetRegistrySettings@CESDHCBase@@QAAHPAVCReg@@@Z 1000551c f   bspesdhc.obj
 0001:00004734       ?BspESDHCGetBaseClk@CESDHCBase@@QAAKXZ 10005734 f   bspesdhc.obj
 0001:000047c0       ?BspESDHCInit@CESDHCBase@@QAAHXZ 100057c0 f   bspesdhc.obj
 0001:00004c90       ?BspESDHCDeinit@CESDHCBase@@QAAXXZ 10005c90 f   bspesdhc.obj
 0001:00004ca0       ?BspESDHCSysIntrSetup@CESDHCBase@@QAAHXZ 10005ca0 f   bspesdhc.obj
 0001:00004de0       ?BspESDHCSetClockGating@CESDHCBase@@QAAXK@Z 10005de0 f   bspesdhc.obj
 0001:00004f00       ?BspESDHCSetSlotVoltage@CESDHCBase@@QAAXK@Z 10005f00 f   bspesdhc.obj
 0001:00004f10       ?BspESDHCIsCardPresent@CESDHCBase@@QAAHXZ 10005f10 f   bspesdhc.obj
 0001:00005064       ?BspESDHCSlotStatusChanged@CESDHCBase@@QAAHXZ 10006064 f   bspesdhc.obj
 0001:00005140       ?BspESDHCCardDetectInt@CESDHCBase@@QAAXH@Z 10006140 f   bspesdhc.obj
 0001:00005214       ?BspESDHCIsWriteProtected@CESDHCBase@@QAAHXZ 10006214 f   bspesdhc.obj
 0001:000052c0       ?ValueDW@CReg@@QAAKPBGK@Z  100062c0 f i bspesdhc.obj
 0001:0000532c       ??0CESDHCBaseEDMA@@QAA@AAVCESDHCBase@@@Z 1000632c f   bspesdhcdma.obj
 0001:00005370       ??1CESDHCBaseEDMA@@UAA@XZ  10006370 f   bspesdhcdma.obj
 0001:00005398       ?BspEDMAInit@CESDHCBaseEDMA@@QAAHXZ 10006398 f   bspesdhcdma.obj
 0001:000053bc       ?BspEDMAArm@CESDHCBaseEDMA@@QAAHAAU_SD_BUS_REQUEST@@H@Z 100063bc f   bspesdhcdma.obj
 0001:000053e0       ?BspEDMANotifyEvent@CESDHCBaseEDMA@@QAAHAAU_SD_BUS_REQUEST@@W4_DMAEVENT@@@Z 100063e0 f   bspesdhcdma.obj
 0001:00005404       ?BspEDMACheckCompletion@CESDHCBaseEDMA@@QAA?AW4_DMAEVENT@@H@Z 10006404 f   bspesdhcdma.obj
 0001:00005430       ?DmaSelectBit@CESDHCBaseEDMA@@UAAEXZ 10006430 f i bspesdhcdma.obj
 0001:00005454       ??_GCESDHCBaseEDMA@@UAAPAXI@Z 10006454 f i bspesdhcdma.obj
 0001:00005454       ??_ECESDHCBaseEDMA@@UAAPAXI@Z 10006454 f i bspesdhcdma.obj
 0001:00005494       DllEntry                   10006494 f   esdhcbase_common_topaz_v1:sdmain.obj
 0001:0000553c       SHC_Deinit                 1000653c f   esdhcbase_common_topaz_v1:sdmain.obj
 0001:0000560c       SHC_Init                   1000660c f   esdhcbase_common_topaz_v1:sdmain.obj
 0001:000057b0       SHC_Open                   100067b0 f   esdhcbase_common_topaz_v1:sdmain.obj
 0001:000057dc       SHC_Close                  100067dc f   esdhcbase_common_topaz_v1:sdmain.obj
 0001:00005800       SHC_PowerDown              10006800 f   esdhcbase_common_topaz_v1:sdmain.obj
 0001:00005844       SHC_PowerUp                10006844 f   esdhcbase_common_topaz_v1:sdmain.obj
 0001:000058a8       SHC_IOControl              100068a8 f   esdhcbase_common_topaz_v1:sdmain.obj
 0001:000059a4       ??_GCESDHCBase@@QAAPAXI@Z  100069a4 f i esdhcbase_common_topaz_v1:sdmain.obj
 0001:000059e4       SetEvent                   100069e4 f i esdhcbase_common_topaz_v1:sdmain.obj
 0001:00005a18       ??0CESDHCBase@@QAA@XZ      10006a18 f   esdhcbase_common_topaz_v1:esdhc.obj
 0001:00005bec       ?SoftwareReset@CESDHCBase@@QAAXXZ 10006bec f   esdhcbase_common_topaz_v1:esdhc.obj
 0001:00005c50       ?SoftwareResetSDIO@CESDHCBase@@QAAXXZ 10006c50 f   esdhcbase_common_topaz_v1:esdhc.obj
 0001:00005e94       ?SetInterface@CESDHCBase@@QAAXPAU_SD_CARD_INTERFACE@@@Z 10006e94 f   esdhcbase_common_topaz_v1:esdhc.obj
 0001:000060ec       ?EnableSDIOInterrupts@CESDHCBase@@QAAXXZ 100070ec f   esdhcbase_common_topaz_v1:esdhc.obj
 0001:00006174       ?DisableSDIOInterrupts@CESDHCBase@@QAAXXZ 10007174 f   esdhcbase_common_topaz_v1:esdhc.obj
 0001:00006200       ?SetClockRate@CESDHCBase@@QAAXPAK@Z 10007200 f   esdhcbase_common_topaz_v1:esdhc.obj
 0001:0000655c       ?ClockGateOn@CESDHCBase@@QAAXXZ 1000755c f   esdhcbase_common_topaz_v1:esdhc.obj
 0001:000065b0       ?ClockGateOff@CESDHCBase@@QAAXXZ 100075b0 f   esdhcbase_common_topaz_v1:esdhc.obj
 0001:00006600       ?SendCommand@CESDHCBase@@QAAJPAU_SD_BUS_REQUEST@@@Z 10007600 f   esdhcbase_common_topaz_v1:esdhc.obj
 0001:000070c4       ?HandleRemoval@CESDHCBase@@QAAXH@Z 100080c4 f   esdhcbase_common_topaz_v1:esdhc.obj
 0001:000074e4       ?HandleInsertion@CESDHCBase@@QAAXXZ 100084e4 f   esdhcbase_common_topaz_v1:esdhc.obj
 0001:00007600       ?HandleCommandErrors@CESDHCBase@@QAAXXZ 10008600 f   esdhcbase_common_topaz_v1:esdhc.obj
 0001:000077d0       ?HandleDataErrors@CESDHCBase@@QAAXXZ 100087d0 f   esdhcbase_common_topaz_v1:esdhc.obj
 0001:00007b48       ?HandleReadReady@CESDHCBase@@QAAXXZ 10008b48 f   esdhcbase_common_topaz_v1:esdhc.obj
 0001:00007eb8       ?HandleWriteReady@CESDHCBase@@QAAXXZ 10008eb8 f   esdhcbase_common_topaz_v1:esdhc.obj
 0001:00008250       ?HandleTransferComplete@CESDHCBase@@QAAXXZ 10009250 f   esdhcbase_common_topaz_v1:esdhc.obj
 0001:000085ec       ?HandleInterrupts@CESDHCBase@@QAAXXZ 100095ec f   esdhcbase_common_topaz_v1:esdhc.obj
 0001:00008ca8       ?DumpRegisters@CESDHCBase@@QAAXXZ 10009ca8 f   esdhcbase_common_topaz_v1:esdhc.obj
 0001:00009160       ??1CESDHCBase@@QAA@XZ      1000a160 f   esdhcbase_common_topaz_v1:esdhc.obj
 0001:000091e0       ?Init@CESDHCBase@@QAAHPBG@Z 1000a1e0 f   esdhcbase_common_topaz_v1:esdhc.obj
 0001:000095c0       ?FreeHostContext@CESDHCBase@@QAAXHH@Z 1000a5c0 f   esdhcbase_common_topaz_v1:esdhc.obj
 0001:000096d4       ?IOControl@CESDHCBase@@QAAHKPAEK0KPAK@Z 1000a6d4 f   esdhcbase_common_topaz_v1:esdhc.obj
 0001:00009ad8       ?InterpretCapabilities@CESDHCBase@@QAAHXZ 1000aad8 f   esdhcbase_common_topaz_v1:esdhc.obj
 0001:00009c24       ?Stop@CESDHCBase@@QAAJXZ   1000ac24 f   esdhcbase_common_topaz_v1:esdhc.obj
 0001:00009e68       ?Start@CESDHCBase@@QAAJXZ  1000ae68 f   esdhcbase_common_topaz_v1:esdhc.obj
 0001:0000a3f0       ?SlotOptionHandler@CESDHCBase@@QAAJW4_SD_SLOT_OPTION_CODE@@PAXK@Z 1000b3f0 f   esdhcbase_common_topaz_v1:esdhc.obj
 0001:0000a848       ?ControllerIstThread@CESDHCBase@@QAAKXZ 1000b848 f   esdhcbase_common_topaz_v1:esdhc.obj
 0001:0000a9e0       ?BusRequestHandler@CESDHCBase@@QAAJPAU_SD_BUS_REQUEST@@@Z 1000b9e0 f   esdhcbase_common_topaz_v1:esdhc.obj
 0001:0000acf8       ?CancelIoHandler@CESDHCBase@@QAAEPAU_SD_BUS_REQUEST@@@Z 1000bcf8 f   esdhcbase_common_topaz_v1:esdhc.obj
 0001:0000ad1c       ?CommandCompleteHandler@CESDHCBase@@QAAHXZ 1000bd1c f   esdhcbase_common_topaz_v1:esdhc.obj
 0001:0000b0f8       ?IndicateBusRequestComplete@CESDHCBase@@QAAXPAU_SD_BUS_REQUEST@@J@Z 1000c0f8 f   esdhcbase_common_topaz_v1:esdhc.obj
 0001:0000b324       ?SlotAllocDMABuffer@CESDHCBase@@QAAPAXKPAT_LARGE_INTEGER@@E@Z 1000c324 f   esdhcbase_common_topaz_v1:esdhc.obj
 0001:0000b3a8       ?SlotFreeDMABuffer@CESDHCBase@@QAAHKT_LARGE_INTEGER@@PAXE@Z 1000c3a8 f   esdhcbase_common_topaz_v1:esdhc.obj
 0001:0000b438       ?SDHCInitialize@CESDHCBase@@SAJPAU_SDCARD_HC_CONTEXT@@@Z 1000c438 f   esdhcbase_common_topaz_v1:esdhc.obj
 0001:0000b564       ?SDHCDeinitialize@CESDHCBase@@SAJPAU_SDCARD_HC_CONTEXT@@@Z 1000c564 f   esdhcbase_common_topaz_v1:esdhc.obj
 0001:0000b690       ?SDHCCancelIoHandler@CESDHCBase@@SAEPAU_SDCARD_HC_CONTEXT@@KPAU_SD_BUS_REQUEST@@@Z 1000c690 f   esdhcbase_common_topaz_v1:esdhc.obj
 0001:0000b758       ?SDHCBusRequestHandler@CESDHCBase@@SAJPAU_SDCARD_HC_CONTEXT@@KPAU_SD_BUS_REQUEST@@@Z 1000c758 f   esdhcbase_common_topaz_v1:esdhc.obj
 0001:0000b820       ?SDHCSlotOptionHandler@CESDHCBase@@SAJPAU_SDCARD_HC_CONTEXT@@KW4_SD_SLOT_OPTION_CODE@@PAXK@Z 1000c820 f   esdhcbase_common_topaz_v1:esdhc.obj
 0001:0000b8b4       ?TransferIsSDIOSuspend@CESDHCBase@@QAAHEI@Z 1000c8b4 f i esdhcbase_common_topaz_v1:esdhc.obj
 0001:0000b91c       ?TransferIsSDIOAbort@CESDHCBase@@QAAHEI@Z 1000c91c f i esdhcbase_common_topaz_v1:esdhc.obj
 0001:0000b984       ResetEvent                 1000c984 f i esdhcbase_common_topaz_v1:esdhc.obj
 0001:0000b9b8       ?Open@CReg@@QAAHPAUHKEY__@@PBGK@Z 1000c9b8 f i esdhcbase_common_topaz_v1:esdhc.obj
 0001:0000ba24       ??0CReg@@QAA@XZ            1000ca24 f i esdhcbase_common_topaz_v1:esdhc.obj
 0001:0000ba50       ?ZeroEntries@CReg@@AAAXXZ  1000ca50 f i esdhcbase_common_topaz_v1:esdhc.obj
 0001:0000ba9c       ??1CReg@@QAA@XZ            1000ca9c f i esdhcbase_common_topaz_v1:esdhc.obj
 0001:0000bb40       ?Reset@CReg@@QAAXXZ        1000cb40 f i esdhcbase_common_topaz_v1:esdhc.obj
 0001:0000bb88       ??0CESDHCBaseSDMA@@QAA@AAVCESDHCBase@@@Z 1000cb88 f i esdhcbase_common_topaz_v1:esdhc.obj
 0001:0000bc20       ?IsDMACompleted@CESDHCBaseDMA@@UAA?AW4_DMAEVENT@@H@Z 1000cc20 f i esdhcbase_common_topaz_v1:esdhc.obj
 0001:0000bc6c       ?DmaSelectBit@CESDHCBaseSDMA@@UAAEXZ 1000cc6c f i esdhcbase_common_topaz_v1:esdhc.obj
 0001:0000bc90       ??_GCESDHCBaseSDMA@@UAAPAXI@Z 1000cc90 f i esdhcbase_common_topaz_v1:esdhc.obj
 0001:0000bc90       ??_ECESDHCBaseSDMA@@UAAPAXI@Z 1000cc90 f i esdhcbase_common_topaz_v1:esdhc.obj
 0001:0000bcd0       ?ISTStub@CESDHCBase@@SAKPAX@Z 1000ccd0 f i esdhcbase_common_topaz_v1:esdhc.obj
 0001:0000bd08       GetCurrentThread           1000cd08 f i esdhcbase_common_topaz_v1:esdhc.obj
 0001:0000bd20       ??0CESDHCBaseDMA@@QAA@AAVCESDHCBase@@@Z 1000cd20 f   esdhcbase_common_topaz_v1:esdhcdma.obj
 0001:0000be38       ?Init@CESDHCBaseDMA@@UAAHXZ 1000ce38 f   esdhcbase_common_topaz_v1:esdhcdma.obj
 0001:0000c048       ??1CESDHCBaseDMA@@UAA@XZ   1000d048 f   esdhcbase_common_topaz_v1:esdhcdma.obj
 0001:0000c168       ?ReAllocateDMABufferList@CESDHCBaseDMA@@QAAKK@Z 1000d168 f   esdhcbase_common_topaz_v1:esdhcdma.obj
 0001:0000c280       ?CancelDMA@CESDHCBaseDMA@@UAAHXZ 1000d280 f   esdhcbase_common_topaz_v1:esdhcdma.obj
 0001:0000c33c       ?ArmDMA@CESDHCBaseDMA@@UAAHAAU_SD_BUS_REQUEST@@H@Z 1000d33c f   esdhcbase_common_topaz_v1:esdhcdma.obj
 0001:0000c844       ??1CESDHCBaseSDMA@@UAA@XZ  1000d844 f   esdhcbase_common_topaz_v1:esdhcdma.obj
 0001:0000c8ac       ?Init@CESDHCBaseSDMA@@UAAHXZ 1000d8ac f   esdhcbase_common_topaz_v1:esdhcdma.obj
 0001:0000c8ec       ?GetDMABuffer@CESDHCBaseSDMA@@IAAHAAU_SD_BUS_REQUEST@@H@Z 1000d8ec f   esdhcbase_common_topaz_v1:esdhcdma.obj
 0001:0000d4a0       ?ArmDMA@CESDHCBaseSDMA@@UAAHAAU_SD_BUS_REQUEST@@H@Z 1000e4a0 f   esdhcbase_common_topaz_v1:esdhcdma.obj
 0001:0000d68c       ?DMANotifyEvent@CESDHCBaseSDMA@@UAAHAAU_SD_BUS_REQUEST@@W4_DMAEVENT@@@Z 1000e68c f   esdhcbase_common_topaz_v1:esdhcdma.obj
 0001:0000ddec       ?Init@CESDHCBaseEDMA@@UAAHXZ 1000edec f   esdhcbase_common_topaz_v1:esdhcdma.obj
 0001:0000de64       ?GetDMABuffer@CESDHCBaseEDMA@@IAAHAAU_SD_BUS_REQUEST@@H@Z 1000ee64 f   esdhcbase_common_topaz_v1:esdhcdma.obj
 0001:0000ea64       ?ArmDMA@CESDHCBaseEDMA@@UAAHAAU_SD_BUS_REQUEST@@H@Z 1000fa64 f   esdhcbase_common_topaz_v1:esdhcdma.obj
 0001:0000eb04       ?DMANotifyEvent@CESDHCBaseEDMA@@UAAHAAU_SD_BUS_REQUEST@@W4_DMAEVENT@@@Z 1000fb04 f   esdhcbase_common_topaz_v1:esdhcdma.obj
 0001:0000ee44       ?IsDMACompleted@CESDHCBaseEDMA@@UAA?AW4_DMAEVENT@@H@Z 1000fe44 f   esdhcbase_common_topaz_v1:esdhcdma.obj
 0001:0000ee9c       ??0CESDHCBase32BitADMA@@QAA@AAVCESDHCBase@@@Z 1000fe9c f   esdhcbase_common_topaz_v1:esdhcdma.obj
 0001:0000ef8c       ??1CESDHCBase32BitADMA@@UAA@XZ 1000ff8c f   esdhcbase_common_topaz_v1:esdhcdma.obj
 0001:0000f138       ?Init@CESDHCBase32BitADMA@@UAAHXZ 10010138 f   esdhcbase_common_topaz_v1:esdhcdma.obj
 0001:0000f314       ?GetDMABuffer@CESDHCBase32BitADMA@@QAAHAAU_SD_BUS_REQUEST@@H@Z 10010314 f   esdhcbase_common_topaz_v1:esdhcdma.obj
 0001:0001000c       ?ArmDMA@CESDHCBase32BitADMA@@UAAHAAU_SD_BUS_REQUEST@@H@Z 1001100c f   esdhcbase_common_topaz_v1:esdhcdma.obj
 0001:00010514       ?DMANotifyEvent@CESDHCBase32BitADMA@@UAAHAAU_SD_BUS_REQUEST@@W4_DMAEVENT@@@Z 10011514 f   esdhcbase_common_topaz_v1:esdhcdma.obj
 0001:00010840       ??0CESDHCBase32BitADMA2@@QAA@AAVCESDHCBase@@@Z 10011840 f   esdhcbase_common_topaz_v1:esdhcdma.obj
 0001:00010930       ??1CESDHCBase32BitADMA2@@UAA@XZ 10011930 f   esdhcbase_common_topaz_v1:esdhcdma.obj
 0001:00010adc       ?Init@CESDHCBase32BitADMA2@@UAAHXZ 10011adc f   esdhcbase_common_topaz_v1:esdhcdma.obj
 0001:00010cb8       ?GetDMABuffer@CESDHCBase32BitADMA2@@QAAHAAU_SD_BUS_REQUEST@@H@Z 10011cb8 f   esdhcbase_common_topaz_v1:esdhcdma.obj
 0001:0001186c       ?ArmDMA@CESDHCBase32BitADMA2@@UAAHAAU_SD_BUS_REQUEST@@H@Z 1001286c f   esdhcbase_common_topaz_v1:esdhcdma.obj
 0001:00011c70       ?IsEnoughDescTable@CESDHCBase32BitADMA2@@IAAHK@Z 10012c70 f   esdhcbase_common_topaz_v1:esdhcdma.obj
 0001:00011e4c       ?DMANotifyEvent@CESDHCBase32BitADMA2@@UAAHAAU_SD_BUS_REQUEST@@W4_DMAEVENT@@@Z 10012e4c f   esdhcbase_common_topaz_v1:esdhcdma.obj
 0001:000121a8       ??_ECESDHCBaseDMA@@UAAPAXI@Z 100131a8 f i esdhcbase_common_topaz_v1:esdhcdma.obj
 0001:000121a8       ??_GCESDHCBaseDMA@@UAAPAXI@Z 100131a8 f i esdhcbase_common_topaz_v1:esdhcdma.obj
 0001:000121e8       CeGetCacheInfo             100131e8 f i esdhcbase_common_topaz_v1:esdhcdma.obj
 0001:00012238       ?GetDataCacheSize@CESDHCBaseDMA@@IBAKXZ 10013238 f i esdhcbase_common_topaz_v1:esdhcdma.obj
 0001:000122c8       ?GetDMALengthBit@CESDHCBaseSDMA@@IAAKKK@Z 100132c8 f i esdhcbase_common_topaz_v1:esdhcdma.obj
 0001:0001232c       ?DmaSelectBit@CESDHCBase32BitADMA@@UAAEXZ 1001332c f i esdhcbase_common_topaz_v1:esdhcdma.obj
 0001:00012350       ??_ECESDHCBase32BitADMA@@UAAPAXI@Z 10013350 f i esdhcbase_common_topaz_v1:esdhcdma.obj
 0001:00012350       ??_GCESDHCBase32BitADMA@@UAAPAXI@Z 10013350 f i esdhcbase_common_topaz_v1:esdhcdma.obj
 0001:00012390       ?DmaSelectBit@CESDHCBase32BitADMA2@@UAAEXZ 10013390 f i esdhcbase_common_topaz_v1:esdhcdma.obj
 0001:000123b4       ??_GCESDHCBase32BitADMA2@@UAAPAXI@Z 100133b4 f i esdhcbase_common_topaz_v1:esdhcdma.obj
 0001:000123b4       ??_ECESDHCBase32BitADMA2@@UAAPAXI@Z 100133b4 f i esdhcbase_common_topaz_v1:esdhcdma.obj
 0001:000123f4       ?CspESDHCGetBaseAddr@CESDHCBase@@QAAKK@Z 100133f4 f   esdhcbase_mx25_topaz_v1:mx25esdhc.obj
 0001:00012460       ?CspESDHCGetIRQ@CESDHCBase@@QAAKK@Z 10013460 f   esdhcbase_mx25_topaz_v1:mx25esdhc.obj
 0001:000124c4       NKDbgPrintfW               100134c4 f   coredll:COREDLL.dll
 0001:000124d4       RegQueryValueExW           100134d4 f   coredll:COREDLL.dll
 0001:000124e4       KernelIoControl            100134e4 f   coredll:COREDLL.dll
 0001:000124f4       Sleep                      100134f4 f   coredll:COREDLL.dll
 0001:00012504       SetInterruptEvent          10013504 f   coredll:COREDLL.dll
 0001:00012514       DisableThreadLibraryCalls  10013514 f   coredll:COREDLL.dll
 0001:00012524       RegisterDbgZones           10013524 f   coredll:COREDLL.dll
 0001:00012534       EventModify                10013534 f   coredll:COREDLL.dll
 0001:00012544       SetLastError               10013544 f   coredll:COREDLL.dll
 0001:00012554       LocalFree                  10013554 f   coredll:COREDLL.dll
 0001:00012564       LocalAlloc                 10013564 f   coredll:COREDLL.dll
 0001:00012574       CloseHandle                10013574 f   coredll:COREDLL.dll
 0001:00012584       WaitForSingleObject        10013584 f   coredll:COREDLL.dll
 0001:00012594       GetLastError               10013594 f   coredll:COREDLL.dll
 0001:000125a4       CreateEventW               100135a4 f   coredll:COREDLL.dll
 0001:000125b4       RegCloseKey                100135b4 f   coredll:COREDLL.dll
 0001:000125c4       OpenDeviceKey              100135c4 f   coredll:COREDLL.dll
 0001:000125d4       RegOpenKeyExW              100135d4 f   coredll:COREDLL.dll
 0001:000125e4       CeSafeCopyMemory           100135e4 f   coredll:COREDLL.dll
 0001:000125f4       InterruptDisable           100135f4 f   coredll:COREDLL.dll
 0001:00012604       CreateThread               10013604 f   coredll:COREDLL.dll
 0001:00012614       InterruptInitialize        10013614 f   coredll:COREDLL.dll
 0001:00012624       LeaveCriticalSection       10013624 f   coredll:COREDLL.dll
 0001:00012634       EnterCriticalSection       10013634 f   coredll:COREDLL.dll
 0001:00012644       InterruptDone              10013644 f   coredll:COREDLL.dll
 0001:00012654       CeSetThreadPriority        10013654 f   coredll:COREDLL.dll
 0001:00012664       InterruptMask              10013664 f   coredll:COREDLL.dll
 0001:00012674       UnlockPages                10013674 f   coredll:COREDLL.dll
 0001:00012684       CacheRangeFlush            10013684 f   coredll:COREDLL.dll
 0001:00012694       LockPages                  10013694 f   coredll:COREDLL.dll
 0001:000126a4       MmMapIoSpace               100136a4 f   ceddk:CEDDK.dll
 0001:000126b4       MmUnmapIoSpace             100136b4 f   ceddk:CEDDK.dll
 0001:000126c4       OALDMAAllocBuffer          100136c4 f   ceddk:CEDDK.dll
 0001:000126d4       OALDMAFreeBuffer           100136d4 f   ceddk:CEDDK.dll
 0001:000126e4       DMACloseBuffer             100136e4 f   ceddk:CEDDK.dll
 0001:000126f4       DMAGetBufferPhysAddr       100136f4 f   ceddk:CEDDK.dll
 0001:00012704       DMAOpenBuffer              10013704 f   ceddk:CEDDK.dll
 0001:00012714       DDKClockGetFreq            10013714 f   cspddk:CSPDDK.dll
 0001:00012724       DDKIomuxSelectInput        10013724 f   cspddk:CSPDDK.dll
 0001:00012734       DDKGpioSetConfig           10013734 f   cspddk:CSPDDK.dll
 0001:00012744       DDKIomuxSetPadConfig       10013744 f   cspddk:CSPDDK.dll
 0001:00012754       DDKIomuxSetPinMux          10013754 f   cspddk:CSPDDK.dll
 0001:00012764       DDKClockSetGatingMode      10013764 f   cspddk:CSPDDK.dll
 0001:00012774       DDKGpioClearIntrPin        10013774 f   cspddk:CSPDDK.dll
 0001:00012784       DDKGpioReadDataPin         10013784 f   cspddk:CSPDDK.dll
 0001:00012794       DDKGpioReadIntrPin         10013794 f   cspddk:CSPDDK.dll
 0001:000127a4       ??3@YAXPAX@Z               100137a4 f   corelib1:COREDLL.dll
 0001:000127b4       ??2@YAPAXI@Z               100137b4 f   corelib1:COREDLL.dll
 0001:000127c4       __rt_udiv                  100137c4 f   corelib1:COREDLL.dll
 0001:000127d4       __C_specific_handler       100137d4 f   corelib1:COREDLL.dll
 0001:000127e4       memset                     100137e4 f   corelib1:COREDLL.dll
 0001:000127f4       wcsncpy_s                  100137f4 f   corelib1:COREDLL.dll
 0001:00012804       _purecall                  10013804 f   corelib1:COREDLL.dll
 0001:00012814       memcpy                     10013814 f   corelib1:COREDLL.dll
 0001:00012824       SDInitializeCardLib        10013824 f   sdcardlib:SDMemApi.obj
 0001:00012990       SDDeinitializeCardLib      10013990 f   sdcardlib:SDMemApi.obj
 0001:00012aec       SDAllocateMemoryWithTag    10013aec f   sdcardlib:SDMemApi.obj
 0001:00012b8c       SDFreeMemory               10013b8c f   sdcardlib:SDMemApi.obj
 0001:00012c10       SDDeleteMemList            10013c10 f   sdcardlib:SDMemApi.obj
 0001:00012db8       SDCreateMemoryList         10013db8 f   sdcardlib:SDMemApi.obj
 0001:00013080       SDFreeToMemList            10014080 f   sdcardlib:SDMemApi.obj
 0001:0001317c       SDAllocateFromMemList      1001417c f   sdcardlib:SDMemApi.obj
 0001:00013294       ??_GCSDMemList@@QAAPAXI@Z  10014294 f i sdcardlib:SDMemApi.obj
 0001:000132d4       ??1CSDMemList@@QAA@XZ      100142d4 f i sdcardlib:SDMemApi.obj
 0001:000132ec       ??0CSDMemList@@QAA@KK@Z    100142ec f i sdcardlib:SDMemApi.obj
 0001:00013330       ?Init@CSDMemList@@QAAHXZ   10014330 f i sdcardlib:SDMemApi.obj
 0001:000133a0       ?Alloc@CSDMemList@@QAAPAXXZ 100143a0 f i sdcardlib:SDMemApi.obj
 0001:000133dc       ?Free@CSDMemList@@QAAXPAX@Z 100143dc f i sdcardlib:SDMemApi.obj
 0001:00013404       ??0?$fixed_block_allocator@$0BE@@ce@@QAA@I@Z 10014404 f i sdcardlib:SDMemApi.obj
 0001:00013434       ??1?$fixed_block_allocator@$0BE@@ce@@QAA@XZ 10014434 f i sdcardlib:SDMemApi.obj
 0001:000134d8       ?allocate@?$fixed_block_allocator@$0BE@@ce@@QBAPAXI@Z 100144d8 f i sdcardlib:SDMemApi.obj
 0001:000135fc       ?deallocate@?$fixed_block_allocator@$0BE@@ce@@QBAXPAXI@Z 100145fc f i sdcardlib:SDMemApi.obj
 0001:00013690       ?_Initialize@?$fixed_block_allocator@$0BE@@ce@@IAAXI@Z 10014690 f i sdcardlib:SDMemApi.obj
 0001:000136e8       ?_InitializeDescr@?$fixed_block_allocator@$0BE@@ce@@IBA_NI@Z 100146e8 f i sdcardlib:SDMemApi.obj
 0001:00013818       SDCardDebugOutput          10014818 f   sdcardlib:SDDebug.obj
 0001:000138c4       SDProcessException         100148c4 f   sdcardlib:SDDebug.obj
 0001:00013ed0       SDPerformSafeCopy          10014ed0 f   sdcardlib:SDDebug.obj
 0001:00013fb8       SDOutputBuffer             10014fb8 f   sdcardlib:SDDebug.obj
 0001:00014440       SDRegisterDebugZones       10015440 f   sdcardlib:SDCardApiStubs.obj
 0001:00014450       SDRegisterClient           10015450 f   sdcardlib:SDCardApiStubs.obj
 0001:00014874       IsKModeAddr                10015874 f i sdcardlib:SDCardApiStubs.obj
 0001:000148b8       svsutil_Initialize         100158b8 f   sdcardlib:utilmem.obj
 0001:00014a18       svsutil_DeInitialize       10015a18 f   sdcardlib:utilmem.obj
 0001:00014ad8       svsutil_TotalAlloc         10015ad8 f   sdcardlib:utilmem.obj
 0001:00014af8       svsutil_LogCallStack       10015af8 f   sdcardlib:utilmem.obj
 0001:00014afc       svsutil_Alloc              10015afc f   sdcardlib:utilmem.obj
 0001:00014d20       svsutil_ReAlloc            10015d20 f   sdcardlib:utilmem.obj
 0001:00015030       svsutil_Free               10016030 f   sdcardlib:utilmem.obj
 0001:0001532c       svsutil_SetAlloc           1001632c f   sdcardlib:utilmem.obj
 0001:000153ac       svsutil_SetAllocData       100163ac f   sdcardlib:utilmem.obj
 0001:000153dc       ?ULongAdd@@YAJKKPAK@Z      100163dc f i sdcardlib:utilmem.obj
 0001:0001544c       svsutil_AllocFixedMemDescrSynch 1001644c f   sdcardlib:utilmemf.obj
 0001:00015590       svsutil_AllocFixedMemDescr 10016590 f   sdcardlib:utilmemf.obj
 0001:000155c8       svsutil_IsFixedEmpty       100165c8 f   sdcardlib:utilmemf.obj
 0001:00015614       svsutil_FixedBlockSize     10016614 f   sdcardlib:utilmemf.obj
 0001:00015640       svsutil_GetFixed           10016640 f   sdcardlib:utilmemf.obj
 0001:000157f4       svsutil_FreeFixed          100167f4 f   sdcardlib:utilmemf.obj
 0001:00015970       svsutil_ReleaseFixedNonEmpty 10016970 f   sdcardlib:utilmemf.obj
 0001:00015a3c       svsutil_ReleaseFixedEmpty  10016a3c f   sdcardlib:utilmemf.obj
 0001:00015b60       svsutil_CompactFixed       10016b60 f   sdcardlib:utilmemf.obj
 0001:00016120       svsutil_GetFixedStats      10017120 f   sdcardlib:utilmemf.obj
 0001:00016238       ??0SVSLocalCriticalSectionX@@QAA@PAUCRITICAL_SECTION@@@Z 10017238 f i sdcardlib:utilmemf.obj
 0001:00016284       ??1SVSLocalCriticalSectionX@@QAA@XZ 10017284 f i sdcardlib:utilmemf.obj
 0001:000162b0       ?LocateLeftNeighbor@SVSTree@@QAAPAVSVSTNode@@K@Z 100172b0 f i sdcardlib:utilmemf.obj
 0001:000163dc       ?Prev@SVSTree@@QAAPAVSVSTNode@@PAV2@@Z 100173dc f i sdcardlib:utilmemf.obj
 0001:000164f8       ?GetData@SVSTree@@SAPAXPAVSVSTNode@@@Z 100174f8 f i sdcardlib:utilmemf.obj
 0001:00016524       ?SVSNewTree@@YAPAVSVSTree@@I@Z 10017524 f i sdcardlib:utilmemf.obj
 0001:00016610       ??2SVSAllocClass@@SAPAXI@Z 10017610 f i sdcardlib:utilmemf.obj
 0001:00016694       ?IsTreeInitialized@SVSTree@@QAAHXZ 10017694 f i sdcardlib:utilmemf.obj
 0001:000166e0       ??0SVSTree@@QAA@I@Z        100176e0 f i sdcardlib:utilmemf.obj
 0001:000168b0       ?InitializeMembers@SVSTree@@IAAXXZ 100178b0 f i sdcardlib:utilmemf.obj
 0001:00016910       ?EnumStart@SVSTree@@UAAKXZ 10017910 f i sdcardlib:utilmemf.obj
 0001:00016940       ?Min@SVSTree@@QAAPAVSVSTNode@@XZ 10017940 f i sdcardlib:utilmemf.obj
 0001:000169cc       ?EnumNext@SVSTree@@UAAKK@Z 100179cc f i sdcardlib:utilmemf.obj
 0001:00016a00       ?Next@SVSTree@@QAAPAVSVSTNode@@PAV2@@Z 10017a00 f i sdcardlib:utilmemf.obj
 0001:00016b1c       ?EnumGetData@SVSTree@@UAAPAXK@Z 10017b1c f i sdcardlib:utilmemf.obj
 0001:00016b4c       ?EnumGetKey@SVSTree@@UAAKK@Z 10017b4c f i sdcardlib:utilmemf.obj
 0001:00016b7c       ?GetKey@SVSTree@@SAKPAVSVSTNode@@@Z 10017b7c f i sdcardlib:utilmemf.obj
 0001:00016ba4       ??0SVSEnumClass@@QAA@XZ    10017ba4 f i sdcardlib:utilmemf.obj
 0001:00016bd8       ??_GSVSTree@@QAAPAXI@Z     10017bd8 f i sdcardlib:utilmemf.obj
 0001:00016c18       ??3SVSAllocClass@@SAXPAX@Z 10017c18 f i sdcardlib:utilmemf.obj
 0001:00016c48       ??1SVSTree@@QAA@XZ         10017c48 f i sdcardlib:utilmemf.obj
 0001:00016cc8       ?Empty@SVSTree@@QAAXXZ     10017cc8 f i sdcardlib:utilmemf.obj
 0001:00016d1c       ?DeleteSubtree@SVSTree@@IAAXPAVSVSTNode@@@Z 10017d1c f i sdcardlib:utilmemf.obj
 0001:00016d84       ?CreateSDBusAcess@@YAPAVSDBusAccess@@PBG@Z 10017d84 f   sdcardlib:busacc.obj
 0001:00016e8c       ??0SDBusAccess@@QAA@PBG@Z  10017e8c f   sdcardlib:busacc.obj
 0001:00016fdc       ??1SDBusAccess@@QAA@XZ     10017fdc f   sdcardlib:busacc.obj
 0001:00017034       ?Init@SDBusAccess@@QAAHXZ  10018034 f   sdcardlib:busacc.obj
 0001:00017094       ?SDBusCallback@SDBusAccess@@CAHKPAXK0KPAKPAU_OVERLAPPED@@@Z 10018094 f   sdcardlib:busacc.obj
 0001:000172a4       ?SDRegisterClient__X@SDBusAccess@@CAJPAX0PAU_SDCARD_CLIENT_REGISTRATION_INFO@@@Z 100182a4 f   sdcardlib:busacc.obj
 0001:0001741c       ?SDSynchronousBusRequest__X@SDBusAccess@@CAJPAXEKW4SD_TRANSFER_CLASS@@W4_SD_RESPONSE_TYPE@@PAU_SD_COMMAND_RESPONSE@@KKPAEKKPAU__PHYS_BUFF_LIST@@@Z 1001841c f   sdcardlib:busacc.obj
 0001:000175a8       ?SDBusRequestResponse__X@SDBusAccess@@CAJPAXPAU_SD_COMMAND_RESPONSE@@@Z 100185a8 f   sdcardlib:busacc.obj
 0001:000176f0       ?SDBusRequest__X@SDBusAccess@@CAJPAXEKW4SD_TRANSFER_CLASS@@W4_SD_RESPONSE_TYPE@@KKPAEP6AX0PAU_SD_BUS_REQUEST@@0K@ZKPAPAU4@KKPAU__PHYS_BUFF_LIST@@@Z 100186f0 f   sdcardlib:busacc.obj
 0001:000178a4       ?SDCancelBusRequest__X@SDBusAccess@@CAEPAU_SD_BUS_REQUEST@@@Z 100188a4 f   sdcardlib:busacc.obj
 0001:0001799c       ?SDFreeBusRequest__X@SDBusAccess@@CAXPAU_SD_BUS_REQUEST@@@Z 1001899c f   sdcardlib:busacc.obj
 0001:00017a6c       ?SDCardInfoQuery__X@SDBusAccess@@CAJPAXW4SD_INFO_TYPE@@0K@Z 10018a6c f   sdcardlib:busacc.obj
 0001:00017b94       ?SDReadWriteRegistersDirect__X@SDBusAccess@@CAJPAXW4SD_IO_TRANSFER_TYPE@@EKEPAEK@Z 10018b94 f   sdcardlib:busacc.obj
 0001:00017ce4       ?SDGetTuple__X@SDBusAccess@@CAJPAXEPAEPAKH@Z 10018ce4 f   sdcardlib:busacc.obj
 0001:00017e5c       ?SDIOConnectInterrupt__X@SDBusAccess@@CAJPAXP6AJ00@Z@Z 10018e5c f   sdcardlib:busacc.obj
 0001:00017f94       ?SDIODisconnectInterrupt__X@SDBusAccess@@CAXPAX@Z 10018f94 f   sdcardlib:busacc.obj
 0001:00018064       ?SDSetCardFeature__X@SDBusAccess@@CAJPAXW4SD_SET_FEATURE_TYPE@@0K@Z 10019064 f   sdcardlib:busacc.obj
 0001:0001819c       SDBusGetClientFunctions    1001919c f   sdcardlib:busacc.obj
 0001:00018224       GetBusAccessHandle         10019224 f   sdcardlib:busacc.obj
 0001:00018278       ??_GSDBusAccess@@QAAPAXI@Z 10019278 f i sdcardlib:busacc.obj
 0001:000182b8       ?GetCallbackHandle@SDBusAccess@@QAAPAXXZ 100192b8 f i sdcardlib:busacc.obj
 0001:000182e4       ?GetBusAccessHandle@SDBusAccess@@QAAPAXXZ 100192e4 f i sdcardlib:busacc.obj
 0001:0001839c       svsutil_AssertBroken       1001939c f   sdcardlib:svsutil.obj
 0001:000183f0       svsutil_wcsdup             100193f0 f   sdcardlib:svsutil.obj
 0001:00018488       svsutil_strdup             10019488 f   sdcardlib:svsutil.obj
 0001:00018518       svsutil_OpenAndReadFile    10019518 f   sdcardlib:svsutil.obj
 0001:00018708       ?svsutil_ReportEventPrintf@@YAHPAXGPAGZZ 10019708 f   sdcardlib:svsutil.obj
 0001:0001880c       ?svsutil_ReportEventPrintfRC@@YAHPAXPAUHINSTANCE__@@KGZZ 1001980c f   sdcardlib:svsutil.obj
 0001:00018950       ??$_vsnwprintf_s@$0IA@@@YAHAAY0IA@GIPBGPAD@Z 10019950 f i sdcardlib:svsutil.obj
 0001:00018994       svsutil_GetTree            10019994 f   sdcardlib:utiltree.obj
 0001:000189c4       svsutil_EmptyTree          100199c4 f   sdcardlib:utiltree.obj
 0001:00018a14       svsutil_EmptyTreeWithCallback 10019a14 f   sdcardlib:utiltree.obj
 0001:00018a78       svsutil_DestroyTree        10019a78 f   sdcardlib:utiltree.obj
 0001:00018b00       svsutil_NextTreeNode       10019b00 f   sdcardlib:utiltree.obj
 0001:00018b70       svsutil_PrevTreeNode       10019b70 f   sdcardlib:utiltree.obj
 0001:00018be0       svsutil_MinTreeNode        10019be0 f   sdcardlib:utiltree.obj
 0001:00018c40       svsutil_MaxTreeNode        10019c40 f   sdcardlib:utiltree.obj
 0001:00018ca0       svsutil_LocateTreeNode     10019ca0 f   sdcardlib:utiltree.obj
 0001:00018d04       svsutil_LocateLeftNeighborNode 10019d04 f   sdcardlib:utiltree.obj
 0001:00018d68       ?svsutil_LocateRightNeighborNode@@YAPAVSVSTNode@@PAVSVSTree@@K@Z 10019d68 f   sdcardlib:utiltree.obj
 0001:00018dcc       svsutil_TreeToArray        10019dcc f   sdcardlib:utiltree.obj
 0001:00018e30       svsutil_GetTreeSize        10019e30 f   sdcardlib:utiltree.obj
 0001:00018e90       svsutil_InsertTreeNode     10019e90 f   sdcardlib:utiltree.obj
 0001:00018ef8       svsutil_DeleteTreeNode     10019ef8 f   sdcardlib:utiltree.obj
 0001:00018f68       svsutil_GetTreeNodeData    10019f68 f   sdcardlib:utiltree.obj
 0001:00018fc8       svsutil_GetTreeNodeKey     10019fc8 f   sdcardlib:utiltree.obj
 0001:00019028       svsutil_CompactTree        1001a028 f   sdcardlib:utiltree.obj
 0001:00019078       ?Insert@SVSTree@@QAAPAVSVSTNode@@KPAX@Z 1001a078 f   sdcardlib:utiltree.obj
 0001:0001941c       ?DeleteFixup@SVSTree@@IAAXPAVSVSTNode@@@Z 1001a41c f   sdcardlib:utiltree.obj
 0001:00019808       ?Delete@SVSTree@@QAAPAXPAVSVSTNode@@@Z 1001a808 f   sdcardlib:utiltree.obj
 0001:00019c04       ?RBTreeIntegrity@SVSTree@@IAAXXZ 1001ac04 f   sdcardlib:utiltree.obj
 0001:0001a01c       ?CheckBlackHeight@SVSTree@@IAAHPAVSVSTNode@@@Z 1001b01c f   sdcardlib:utiltree.obj
 0001:0001a264       ?InTree@SVSTree@@IAAHPAVSVSTNode@@@Z 1001b264 f   sdcardlib:utiltree.obj
 0001:0001a2f8       ?Empty@SVSTree@@QAAXP6AXPAX0@Z0@Z 1001b2f8 f i sdcardlib:utiltree.obj
 0001:0001a354       ?DeleteSubtree@SVSTree@@IAAXPAVSVSTNode@@P6AXPAX1@Z1@Z 1001b354 f i sdcardlib:utiltree.obj
 0001:0001a3e4       ?Max@SVSTree@@QAAPAVSVSTNode@@XZ 1001b3e4 f i sdcardlib:utiltree.obj
 0001:0001a470       ?Locate@SVSTree@@QAAPAVSVSTNode@@K@Z 1001b470 f i sdcardlib:utiltree.obj
 0001:0001a530       ?LocateRightNeighbor@SVSTree@@QAAPAVSVSTNode@@K@Z 1001b530 f i sdcardlib:utiltree.obj
 0001:0001a65c       ?ToArray@SVSTree@@QAAIPAPAX@Z 1001b65c f i sdcardlib:utiltree.obj
 0001:0001a69c       ?SubtreeToArray@SVSTree@@IAAIPAVSVSTNode@@AAPAPAX@Z 1001b69c f i sdcardlib:utiltree.obj
 0001:0001a7a4       ?Size@SVSTree@@QAAIXZ      1001b7a4 f i sdcardlib:utiltree.obj
 0001:0001a7d0       ?Compact@SVSTree@@QAAXXZ   1001b7d0 f i sdcardlib:utiltree.obj
 0001:0001a7f0       ?TreeInsert@SVSTree@@IAAXPAVSVSTNode@@@Z 1001b7f0 f i sdcardlib:utiltree.obj
 0001:0001a91c       ?LeftRotate@SVSTree@@IAAXPAVSVSTNode@@@Z 1001b91c f i sdcardlib:utiltree.obj
 0001:0001aa54       ?RightRotate@SVSTree@@IAAXPAVSVSTNode@@@Z 1001ba54 f i sdcardlib:utiltree.obj
 0001:0001ab8c       SDHCDInitializeHCLib       1001bb8c f   sdhclib:SDHCLib.obj
 0001:0001ae44       SDHCDDeinitializeHCLib     1001be44 f   sdhclib:SDHCLib.obj
 0001:0001ae5c       SDHCDAllocateContext       1001be5c f   sdhclib:SDHCLib.obj
 0001:0001af0c       SDHCDDeleteContext         1001bf0c f   sdhclib:SDHCLib.obj
 0001:0001af80       SDHCDRegisterHostController 1001bf80 f   sdhclib:SDHCLib.obj
 0001:0001b004       SDHCDDeregisterHostController 1001c004 f   sdhclib:SDHCLib.obj
 0001:0001b088       SDHCDIndicateSlotStateChange 1001c088 f   sdhclib:SDHCLib.obj
 0001:0001b104       SDHCDIndicateBusRequestComplete 1001c104 f   sdhclib:SDHCLib.obj
 0001:0001b180       SDHCDUnlockRequest         1001c180 f   sdhclib:SDHCLib.obj
 0001:0001b1f8       SDHCDGetAndLockCurrentRequest 1001c1f8 f   sdhclib:SDHCLib.obj
 0001:0001b280       SDHCDPowerUpDown           1001c280 f   sdhclib:SDHCLib.obj
 0001:0001b300       SDHCDGetHCFunctions        1001c300 f   sdbus:SDBus.dll
 0001:0001b310       InterlockedDecrement       1001c310 f   coredll:COREDLL.dll
 0001:0001b320       InterlockedIncrement       1001c320 f   coredll:COREDLL.dll
 0001:0001b330       DeleteCriticalSection      1001c330 f   coredll:COREDLL.dll
 0001:0001b340       InitializeCriticalSection  1001c340 f   coredll:COREDLL.dll
 0001:0001b350       InterlockedCompareExchange 1001c350 f   coredll:COREDLL.dll
 0001:0001b360       OutputDebugStringW         1001c360 f   coredll:COREDLL.dll
 0001:0001b370       StringCchVPrintfW          1001c370 f   coredll:COREDLL.dll
 0001:0001b380       StringCchCatW              1001c380 f   coredll:COREDLL.dll
 0001:0001b390       StringCchCopyW             1001c390 f   coredll:COREDLL.dll
 0001:0001b3a0       StringCchPrintfW           1001c3a0 f   coredll:COREDLL.dll
 0001:0001b3b0       InterlockedExchange        1001c3b0 f   coredll:COREDLL.dll
 0001:0001b3c0       ReadFile                   1001c3c0 f   coredll:COREDLL.dll
 0001:0001b3d0       GetFileSize                1001c3d0 f   coredll:COREDLL.dll
 0001:0001b3e0       CreateFileW                1001c3e0 f   coredll:COREDLL.dll
 0001:0001b3f0       ReportEventW               1001c3f0 f   coredll:COREDLL.dll
 0001:0001b400       LoadStringW                1001c400 f   coredll:COREDLL.dll
 0001:0001b410       BusIoControl               1001c410 f   ceddk:CEDDK.dll
 0001:0001b420       CeDriverMapCallbackFunction 1001c420 f   ceddk:CEDDK.dll
 0001:0001b430       CreateBusAccessHandle      1001c430 f   ceddk:CEDDK.dll
 0001:0001b440       CloseBusAccessHandle       1001c440 f   ceddk:CEDDK.dll
 0001:0001b450       __security_init_cookie     1001c450 f   corelib0:seccinit.obj
 0001:0001b4e8       __GSHandlerCheck           1001c4e8 f   corelib0:gshandler.obj
 0001:0001b52c       __GSHandlerCheckCommon     1001c52c f   corelib0:gshandler.obj
 0001:0001b5d0       __security_check_cookie    1001c5d0 f   corelib0:armsecgs.obj
 0001:0001b5e0       __gsfailure                1001c5e0     corelib0:armsecgs.obj
 0001:0001b624       __GSHandlerCheck_SEH       1001c624 f   corelib0:gshandlerseh.obj
 0001:0001b6a8       malloc                     1001c6a8 f   corelib1:COREDLL.dll
 0001:0001b6b8       realloc                    1001c6b8 f   corelib1:COREDLL.dll
 0001:0001b6c8       free                       1001c6c8 f   corelib1:COREDLL.dll
 0001:0001b6d8       wcslen                     1001c6d8 f   corelib1:COREDLL.dll
 0001:0001b6e8       strlen                     1001c6e8 f   corelib1:COREDLL.dll
 0001:0001b6f8       _vsnwprintf_s              1001c6f8 f   corelib1:COREDLL.dll
 0001:0001b708       __security_gen_cookie2     1001c708 f   corelib1:COREDLL.dll
 0001:0001b718       __report_gsfailure         1001c718 f   corelib1:COREDLL.dll
 0001:0001b790       __IMPORT_DESCRIPTOR_COREDLL 1001c790     coredll:COREDLL.dll
 0001:0001b7a4       __IMPORT_DESCRIPTOR_CEDDK  1001c7a4     ceddk:CEDDK.dll
 0001:0001b7b8       __IMPORT_DESCRIPTOR_CSPDDK 1001c7b8     cspddk:CSPDDK.dll
 0001:0001b7cc       __IMPORT_DESCRIPTOR_SDBus  1001c7cc     sdbus:SDBus.dll
 0001:0001b7e0       __NULL_IMPORT_DESCRIPTOR   1001c7e0     coredll:COREDLL.dll
 0002:00000000       __imp_BusIoControl         1001d000     ceddk:CEDDK.dll
 0002:00000004       __imp_CreateBusAccessHandle 1001d004     ceddk:CEDDK.dll
 0002:00000008       __imp_CloseBusAccessHandle 1001d008     ceddk:CEDDK.dll
 0002:0000000c       __imp_DMAOpenBuffer        1001d00c     ceddk:CEDDK.dll
 0002:00000010       __imp_DMAGetBufferPhysAddr 1001d010     ceddk:CEDDK.dll
 0002:00000014       __imp_DMACloseBuffer       1001d014     ceddk:CEDDK.dll
 0002:00000018       __imp_OALDMAFreeBuffer     1001d018     ceddk:CEDDK.dll
 0002:0000001c       __imp_OALDMAAllocBuffer    1001d01c     ceddk:CEDDK.dll
 0002:00000020       __imp_MmUnmapIoSpace       1001d020     ceddk:CEDDK.dll
 0002:00000024       __imp_MmMapIoSpace         1001d024     ceddk:CEDDK.dll
 0002:00000028       __imp_CeDriverMapCallbackFunction 1001d028     ceddk:CEDDK.dll
 0002:0000002c       \177CEDDK_NULL_THUNK_DATA  1001d02c     ceddk:CEDDK.dll
 0002:00000030       __imp_WaitForSingleObject  1001d030     coredll:COREDLL.dll
 0002:00000034       __imp_GetLastError         1001d034     coredll:COREDLL.dll
 0002:00000038       __imp_CreateEventW         1001d038     coredll:COREDLL.dll
 0002:0000003c       __imp_RegCloseKey          1001d03c     coredll:COREDLL.dll
 0002:00000040       __imp_OpenDeviceKey        1001d040     coredll:COREDLL.dll
 0002:00000044       __imp_RegOpenKeyExW        1001d044     coredll:COREDLL.dll
 0002:00000048       __imp_CeSafeCopyMemory     1001d048     coredll:COREDLL.dll
 0002:0000004c       __imp_InterruptDisable     1001d04c     coredll:COREDLL.dll
 0002:00000050       __imp_CreateThread         1001d050     coredll:COREDLL.dll
 0002:00000054       __imp_InterruptInitialize  1001d054     coredll:COREDLL.dll
 0002:00000058       __imp_LeaveCriticalSection 1001d058     coredll:COREDLL.dll
 0002:0000005c       __imp_EnterCriticalSection 1001d05c     coredll:COREDLL.dll
 0002:00000060       __imp_InterruptDone        1001d060     coredll:COREDLL.dll
 0002:00000064       __imp_CeSetThreadPriority  1001d064     coredll:COREDLL.dll
 0002:00000068       __imp_InterruptMask        1001d068     coredll:COREDLL.dll
 0002:0000006c       __imp_UnlockPages          1001d06c     coredll:COREDLL.dll
 0002:00000070       __imp_CacheRangeFlush      1001d070     coredll:COREDLL.dll
 0002:00000074       __imp_CloseHandle          1001d074     coredll:COREDLL.dll
 0002:00000078       __imp_LocalAlloc           1001d078     coredll:COREDLL.dll
 0002:0000007c       __imp_LocalFree            1001d07c     coredll:COREDLL.dll
 0002:00000080       __imp_SetLastError         1001d080     coredll:COREDLL.dll
 0002:00000084       __imp_EventModify          1001d084     coredll:COREDLL.dll
 0002:00000088       __imp_RegisterDbgZones     1001d088     coredll:COREDLL.dll
 0002:0000008c       __imp_DisableThreadLibraryCalls 1001d08c     coredll:COREDLL.dll
 0002:00000090       __imp_SetInterruptEvent    1001d090     coredll:COREDLL.dll
 0002:00000094       __imp_Sleep                1001d094     coredll:COREDLL.dll
 0002:00000098       __imp___security_gen_cookie2 1001d098     corelib1:COREDLL.dll
 0002:0000009c       __imp__vsnwprintf_s        1001d09c     corelib1:COREDLL.dll
 0002:000000a0       __imp_strlen               1001d0a0     corelib1:COREDLL.dll
 0002:000000a4       __imp_wcslen               1001d0a4     corelib1:COREDLL.dll
 0002:000000a8       __imp___report_gsfailure   1001d0a8     corelib1:COREDLL.dll
 0002:000000ac       __imp_free                 1001d0ac     corelib1:COREDLL.dll
 0002:000000b0       __imp_realloc              1001d0b0     corelib1:COREDLL.dll
 0002:000000b4       __imp_malloc               1001d0b4     corelib1:COREDLL.dll
 0002:000000b8       __imp_KernelIoControl      1001d0b8     coredll:COREDLL.dll
 0002:000000bc       __imp_RegQueryValueExW     1001d0bc     coredll:COREDLL.dll
 0002:000000c0       __imp_??3@YAXPAX@Z         1001d0c0     corelib1:COREDLL.dll
 0002:000000c4       __imp_??2@YAPAXI@Z         1001d0c4     corelib1:COREDLL.dll
 0002:000000c8       __imp___rt_udiv            1001d0c8     corelib1:COREDLL.dll
 0002:000000cc       __imp___C_specific_handler 1001d0cc     corelib1:COREDLL.dll
 0002:000000d0       __imp_memset               1001d0d0     corelib1:COREDLL.dll
 0002:000000d4       __imp_wcsncpy_s            1001d0d4     corelib1:COREDLL.dll
 0002:000000d8       __imp__purecall            1001d0d8     corelib1:COREDLL.dll
 0002:000000dc       __imp_memcpy               1001d0dc     corelib1:COREDLL.dll
 0002:000000e0       __imp_LockPages            1001d0e0     coredll:COREDLL.dll
 0002:000000e4       __imp_NKDbgPrintfW         1001d0e4     coredll:COREDLL.dll
 0002:000000e8       __imp_InterlockedDecrement 1001d0e8     coredll:COREDLL.dll
 0002:000000ec       __imp_InterlockedIncrement 1001d0ec     coredll:COREDLL.dll
 0002:000000f0       __imp_DeleteCriticalSection 1001d0f0     coredll:COREDLL.dll
 0002:000000f4       __imp_InitializeCriticalSection 1001d0f4     coredll:COREDLL.dll
 0002:000000f8       __imp_InterlockedCompareExchange 1001d0f8     coredll:COREDLL.dll
 0002:000000fc       __imp_OutputDebugStringW   1001d0fc     coredll:COREDLL.dll
 0002:00000100       __imp_StringCchVPrintfW    1001d100     coredll:COREDLL.dll
 0002:00000104       __imp_StringCchCatW        1001d104     coredll:COREDLL.dll
 0002:00000108       __imp_StringCchCopyW       1001d108     coredll:COREDLL.dll
 0002:0000010c       __imp_StringCchPrintfW     1001d10c     coredll:COREDLL.dll
 0002:00000110       __imp_InterlockedExchange  1001d110     coredll:COREDLL.dll
 0002:00000114       __imp_ReadFile             1001d114     coredll:COREDLL.dll
 0002:00000118       __imp_GetFileSize          1001d118     coredll:COREDLL.dll
 0002:0000011c       __imp_CreateFileW          1001d11c     coredll:COREDLL.dll
 0002:00000120       __imp_ReportEventW         1001d120     coredll:COREDLL.dll
 0002:00000124       __imp_LoadStringW          1001d124     coredll:COREDLL.dll
 0002:00000128       \177COREDLL_NULL_THUNK_DATA 1001d128     coredll:COREDLL.dll
 0002:0000012c       __imp_DDKClockSetGatingMode 1001d12c     cspddk:CSPDDK.dll
 0002:00000130       __imp_DDKClockGetFreq      1001d130     cspddk:CSPDDK.dll
 0002:00000134       __imp_DDKGpioReadIntrPin   1001d134     cspddk:CSPDDK.dll
 0002:00000138       __imp_DDKGpioReadDataPin   1001d138     cspddk:CSPDDK.dll
 0002:0000013c       __imp_DDKGpioClearIntrPin  1001d13c     cspddk:CSPDDK.dll
 0002:00000140       __imp_DDKIomuxSetPinMux    1001d140     cspddk:CSPDDK.dll
 0002:00000144       __imp_DDKIomuxSetPadConfig 1001d144     cspddk:CSPDDK.dll
 0002:00000148       __imp_DDKGpioSetConfig     1001d148     cspddk:CSPDDK.dll
 0002:0000014c       __imp_DDKIomuxSelectInput  1001d14c     cspddk:CSPDDK.dll
 0002:00000150       \177CSPDDK_NULL_THUNK_DATA 1001d150     cspddk:CSPDDK.dll
 0002:00000154       __imp_SDHCDGetHCFunctions  1001d154     sdbus:SDBus.dll
 0002:00000158       \177SDBus_NULL_THUNK_DATA  1001d158     sdbus:SDBus.dll
 0002:00000168       dpCurSettings              1001d168     esdhcbase_common_topaz_v1:sdmain.obj
 0002:000005ac       g_SDClientApiFunctions     1001d5ac     sdcardlib:SDCardApiStubs.obj
 0002:000005e0       g_funcAlloc                1001d5e0     sdcardlib:utilmem.obj
 0002:000005e4       g_funcFree                 1001d5e4     sdcardlib:utilmem.obj
 0002:000005e8       g_funcRealloc              1001d5e8     sdcardlib:utilmem.obj
 0002:000005ec       g_funcDebugOut             1001d5ec     sdcardlib:svsutil.obj
 0002:000005f0       __security_cookie          1001d5f0     corelib0:seccinit.obj
 0002:000005f4       __security_cookie_complement 1001d5f4     corelib0:seccinit.obj
 0002:00000604       g_pvAllocData              1001d604     sdcardlib:utilmem.obj
 0002:00000608       g_pvFreeData               1001d608     sdcardlib:utilmem.obj
 0002:00000620       ?g_pSDBusAccess@@3PAVSDBusAccess@@A 1001d620     sdcardlib:busacc.obj
 0002:00000624       g_pvDebugData              1001d624     sdcardlib:svsutil.obj

 entry point at        0001:00005494

 Static symbols

 0001:0000734c       ?DumpRequest@@YAXPAU_SD_BUS_REQUEST@@K@Z 1000834c f   esdhcbase_common_topaz_v1:esdhc.obj
 0001:00012908       ?InitCardLib@@YAHXZ        10013908 f   sdcardlib:SDMemApi.obj
 0001:00012a74       ?DeinitCardLib@@YAHXZ      10013a74 f   sdcardlib:SDMemApi.obj
 0001:00018318       ?svsutil_DebugOut@@YAHPAXPAGZZ 10019318 f   sdcardlib:svsutil.obj
